:100000000C9438070C9460070C9460070C946007FC
:100010000C9460070C9460070C9460070C946007C4
:100020000C9460070C9464090C9413330C948B3378
:100030000C9460070C9460070C9460070C946007A4
:100040000C94460E0C9460070C9460070C946007A7
:100050000C9460070C9460070C9460070C94802A41
:100060000C9460070C94522F0C948D2F0C94600705
:100070000C9460070C9460070C9460070C94600764
:100080000C9460070C9460070C9460070C94600754
:100090000C9460070C9460070C9460070C94600744
:1000A0000C9460070C9460070C946007E61DED1D2E
:1000B000ED1DE61DED1DED1DED1DED1DED1DED1DF7
:1000C000ED1DED1DED1DED1DED1DED1DED1D5B1D72
:1000D000ED1DED1DED1DED1DED1DBE1CED1DED1D00
:1000E000ED1DED1DED1DED1DED1DED1DED1DED1DC0
:1000F000ED1DED1DED1DED1DED1D671D671D671D42
:10010000671D671D671D671D671D671DED1DED1DC3
:10011000ED1DED1DED1DED1DC31C661D661D661D4F
:10012000661DED1D771D7F1D871D8F1D971D9F1D52
:10013000A71DAF1DB91DC31DCD1DD71D0A1DCA1C8E
:10014000ED1DED1DED1DED1D5B1DED1DED1DED1DF1
:10015000ED1DED1DED1DED1DED1D651D651D651DE7
:10016000651DED1D771D7F1D871D8F1D971D9F1D13
:10017000A71DAF1DB91DC31DCD1DD71D0A1DCA1C4E
:10018000ED1DED1DED1DED1D5B1D1E1E1E1E1E1E1B
:100190001E1E1E1E1E1E1E1E1E1E1E1E1E1E1E1E7F
:1001A0001E1E1E1E3F1F3F1F3F1F3F1F3F1F3F1FA3
:1001B000651E6F1E791E831EE91EF31E011F131F8D
:1001C000B01F2020F11FF61FFB1F002005200A2072
:1001D0000F2020201A203A274F275B2764277127FA
:1001E00097279F27C227AF27C92BCC2BBF2BC32B09
:1001F000ED2BED2BED2BD02BD42BD82BDE2BE22BA4
:10020000ED2BE82B456E746572206D656E752E2E94
:100210002E00546F67676C6564206D6963726F5060
:10022000504D00546F67676C656420696E76657227
:100230007465642050504D2100546F67676C65648D
:10024000205458206D7574696E672100546F67677C
:100250006C65642074656C656D65747279210050FD
:10026000726F746F636F6C206572726F7220776942
:1002700074682052580054696D656F7574207768F2
:10028000656E20636F6E6E656374696E6720746F50
:1002900020525800507265737320616E79206B652F
:1002A0007920746F2063616E63656C00436F6E6EBE
:1002B000656374696E6720746F2052582C20706FCC
:1002C00077657220757020746865205258202877F1
:1002D0006974682062696E6420706C756720696655
:1002E000206E6F74207573696E6720616C77617919
:1002F000732062696E642900546F67676C656420BF
:1003000027696D6D656469617465206F75747075BA
:10031000742700546F67676C65642027736C61767F
:1003200065206D6F64652700546F67676C65642096
:1003300027616C776179732062696E642700546F5E
:1003400067676C65642050504D206368616E6E6510
:100350006C206C696D697400536574205253534965
:1003600020696E6A656374696F6E206368616E6E82
:10037000656C2028303D3D64697361626C652900BD
:100380005365742050504D206D696E696D756D20F8
:1003900073796E630053657420626561636F6E20CC
:1003A000696E74657276616C005365742062656174
:1003B000636F6E2064656C617900536574206265BB
:1003C00061636F6E206672657175656E6379206911
:1003D0006E20487A3A20303D64697361626C652C06
:1003E0002050783D504D52206368616E6E656C20E0
:1003F000782C2046783D465253206368616E6E65C6
:100400006C2078005365742050574D2073746F70C2
:100410002064656C61792028302064697361626CA6
:1004200065642C20312D323535203D3D20302E3174
:1004300073202D2035306D696E290053657420506E
:10044000504D2073746F702064656C617920283082
:100450002064697361626C65642C20312D323535FE
:10046000203D3D20302E3173202D2035306D696EBA
:100470002900536574206661696C73616665206448
:10048000656C61792028302064697361626C6564F1
:100490002C20312D323535203D3D20302E3173203A
:1004A0002D2035306D696E29002A2A2A2A2A2A2A07
:1004B0002A2A2A2A2A2A2A2A2A2A2A2A2A2A2A2A9C
:1004C0002A2A2A2A2A2A0052582041636B6564206E
:1004D0002D2072657665727420737563636573731E
:1004E00066756C21002A2A2A2A2A2A2A2A2A2A2AD6
:1004F0002A2A2A2A2A2A2A2A2A2A2A2A2A2A2A2A5C
:100500002A2A002A2A2A2A2A2A2A2A2A2A2A2A2A75
:100510002A2A2A2A2A2A2A2A2A2A2A2A2A2A2A2A3B
:100520000052582041636B6564202D207570646112
:100530007465207375636365737366756C21002A37
:100540002A2A2A2A2A2A2A2A2A2A2A2A2A2A2A2A0B
:100550002A2A2A2A2A2A2A2A2A2A2A2A0056616C80
:1005600069642063686F69636573206172653A200E
:100570005B315D2D5B31365D20286368616E6E6591
:100580006C20312D31362900536574206F757470DD
:10059000757420666F7220706F727420005B585DF6
:1005A0002061626F7274206368616E676573206199
:1005B0006E64206578697420525820636F6E666996
:1005C00067005B535D2073617665207365747469A1
:1005D0006E677320746F205258005B525D20726505
:1005E000766572742052582073657474696E6773EF
:1005F00020746F2064656661756C74730055736553
:10060000206E756D62657273205B312D445D2074C0
:100610006F206564697420706F727473205B452D60
:10062000515D20666F722073657474696E67730024
:10063000202D20726563656976657220636F6E6632
:100640006967757261746F722C20727820737720DD
:10065000000A0A6F70656E4C52536E672000536536
:10066000742073657269616C206261756472617473
:10067000653A200056616C69642063686F69636540
:10068000733A2031202D20342B34202F2032202D7E
:100690002038202F2033202D20382B34202F2034B9
:1006A000202D203132202F2035202D2031322B34A7
:1006B000202F2036202D20313600536574204368CA
:1006C000616E6E656C20636F6E6669673A200053D9
:1006D00065742044617461726174652028302D3224
:1006E000293A200053657420486F70206368616E5A
:1006F0006E656C7320286D61782032342C20736510
:100700007061726174656420627920636F6D6D61E0
:1007100073292076616C69642076616C756573203D
:10072000312D3235353A2000536574206368616E8F
:100730006E656C2073706163696E67202878313054
:100740006B487A293A200053657420524620706F16
:100750007765722028302D37293A200053657420A0
:100760005246206D61676963202868657829206595
:100770002E672E20307844454144463030443A209C
:1007800000536574206261736520667265717565DA
:100790006E63792028696E20487A293A20005B5AD6
:1007A0005D20656E74657220726563656976657239
:1007B00020636F6E66696775726174696F6E20750C
:1007C00074696C79005B465D20646973706C617953
:1007D0002061637475616C206672657175656E6306
:1007E0006965732075736564005B525D2063616C9D
:1007F00063756C6174652072616E646F6D206B65EA
:100800007920616E6420686F70206C697374005B7E
:10081000495D207265696E697469616C697A6520E9
:1008200073657474696E677320746F20736B65747D
:1008300063682064656661756C7473005B585D2045
:10084000726576657274206368616E676573206196
:100850006E642065786974206D656E75005B535D0C
:1008600020736176652073657474696E6773207494
:100870006F20454550524F4D20616E642065786968
:1008800074206D656E7500557365206E756D6265BB
:100890007273205B302D395D20746F20656469743C
:1008A00020706172616D657465727300202D205334
:1008B000797374656D20636F6E66696775726174B4
:1008C000696F6E000A0A6F70656E4C52536E672036
:1008D000005129204F7574707574206265666F72BF
:1008E00065206C696E6B20283D465329203A200014
:1008F000502920536C617665206D6F6465202865F2
:1009000078706572696D656E74616C293A20004F6C
:10091000292054696D65642042494E442061742049
:100920007374617274757020203A20004E29205033
:10093000504D206F7574707574206C696D697465A5
:100940006420202020203A200044495341424C4555
:1009500044004D292050504D205253534920746F6C
:10096000206368616E6E656C202020203A20004C68
:10097000292050504D206D696E696D756D20737919
:100980006E63202875732920203A20004449534182
:10099000424C4544004B29204661696C7361666591
:1009A00020626561636F6E20696E74762E20283137
:1009B0002D32353573293A20004A29204661696C69
:1009C0007361666520626561636F6E2064656C614A
:1009D000792028302D323535203D3E2031307320AE
:1009E0002D203135306D696E293A20004929204685
:1009F00061696C7361666520626561636F6E206614
:100A000072712E203A200048292050574D207374CF
:100A10006F702064656C6179202020202020203AAE
:100A2000200047292050504D2073746F702064655A
:100A30006C6179202020202020203A2000462920A7
:100A40004661696C736166652064656C617920201C
:100A500020202020203A200050574D206368616EEE
:100A60006E656C200066756E6374696F6E3A200067
:100A70002920706F72742000506F776572546F7701
:100A8000657200445446205548462033322D626931
:100A9000742031306368004F70656E4C52536E673E
:100AA0005258206D696E6920342F36636800466C99
:100AB0007974726F6E2F4F72616E67655258205550
:100AC00048462038636800525820747970653A208F
:100AD0000044697361626C656400487A00203D3DA2
:100AE000200043616C63756C6174656420706163A0
:100AF0006B657420696E74657276616C3A20004291
:100B000029204D6963726F202868616C6629205026
:100B1000504D202020203A00412920496E766572F0
:100B20007465642050504D20696E20202020203AAA
:100B3000003029204D7574652062757A7A657220BF
:100B4000286D6F73746C79293A00392920536572C6
:100B500069616C2062617564726174653A00736DDD
:100B6000617274506F7274004672536B79005472E4
:100B7000616E73706172656E740044697361626C5A
:100B800065640038292054656C656D657472793A26
:100B900020202020202020003729204368616E6E0D
:100BA000656C20636F6E6669673A202000362920E5
:100BB00044617461726174652028302D32293A20B5
:100BC000202000352920486F70206368616E6E65B3
:100BD0006C733A2020202020003429204368616E65
:100BE0006E656C2073706163696E673A2020003314
:100BF0002920524620706F7765722028302D3729C2
:100C00003A202020003229205246206D6167696316
:100C10003A2020202020202020200031292042615D
:100C20007365206672657175656E63793A20202060
:100C30000000000000240027002A002D00300000E2
:100C4000000000250028002B002E003100000000CD
:100C5000002300260029002C002F000404040404B3
:100C6000030405020202020403020202020606064F
:100C70000606060404020202040408020110408071
:100C80004010204080408008020401804020100273
:100C9000011080102040400000000200080E0000FB
:100CA000030401000B000000000000000000000031
:100CB0000000000000070605040100080A0B0C0DE7
:100CC00009080B00020202010009040000010202EF
:100CD000000005240010010524010101042402067E
:100CE00005240600010705810310004009040100E6
:100CF000020A000000070502024000000705830207
:100D000040000004030904220341007200640075DE
:100D10000069006E006F0020004C0065006F006EDF
:100D2000006100720064006F0018034100720064EB
:100D300000750069006E006F0020004C004C0043FD
:100D40000012010002000000404123368000010132
:100D5000020001120100020200004041233680001F
:100D6000010102000100C18081C105010902A10148
:100D70000901A100850105091901290315002501B3
:100D800095037501810295017505810305010930FF
:100D9000093109381581257F750895038106C0C082
:100DA00005010906A1018502050719E029E71500DB
:100DB0002501750195088102950175088103950645
:100DC0007508150025650507190029658100C0090A
:100DD0000402000103000000092101010001226555
:100DE000000705840340000100000000000000002F
:100DF0002A2B280000000000000000000000000076
:100E000000000000000000002C9EB4A0A1A2A434A9
:100E1000A6A7A5AE362D3738271E1F202122232452
:100E20002526B333B62EB7B89F8485868788898AEE
:100E30008B8C8D8E8F909192939495969798999A8A
:100E40009B9C9D2F3130A3AD350405060708090A88
:100E50000B0C0D0E0F101112131415161718191A6A
:100E60001B1C1DAFB1B0B5009C2C35317132F9346B
:100E700011241FBECFEFDAE0DEBFCDBF13E0A0E04C
:100E8000B1E0E8E8FDE602C005900D92A03CB10794
:100E9000D9F716E0A0ECB3E001C01D92A93EB1075E
:100EA000E1F71EE0C0E7DEE004C02297FE010E94E9
:100EB0009F36C836D107C9F70E947A310C94C236E2
:100EC0000C940000A0E0B0E0E8E6F7E00C946E3689
:100ED000EC01A880B980CA80DB80A114B104C104F0
:100EE000D10441F484E2A82E89EDB82E8BE5C82EFA
:100EF00087E0D82EC601B5012DE133EF41E050E087
:100F00000E944B3627EA31E440E050E00E94F7357A
:100F10007B018C01C601B5012DE133EF41E050E0CA
:100F20000E944B36CA01B9012CEE34EF4FEF5FEF50
:100F30000E94F7356E0D7F1D801F911F97FF04C023
:100F40006150704080409048688379838A839B8396
:100F50009B01AC015F77B901CA01CDB7DEB7EAE00A
:100F60000C948A360E946207089581EB92E00E94F9
:100F7000620708956093B1027093B2028093B30246
:100F80009093B4020895A0E0B0E0E9ECF7E00C948F
:100F90006736EC012B016A016115710519F0FB013F
:100FA00091838083C114D10449F0C60102978397CD
:100FB00028F020E030E040E050E0DCC0A9908A2D2D
:100FC00090E00E94B736892BC9F7FDE2AF1621F4F5
:100FD000A9903324339405C08BE2A81609F4A99094
:100FE0003324C114D10421F0E0E1CE16D10411F56F
:100FF000F0E3AF1669F48881883711F0883541F441
:10100000A980229682E0382A20E1C22ED12C12C07B
:10101000C114D10479F4E0E3AE1659F199E9E92E4F
:1010200099E9F92E99E9092F99E1192F8AE0C82E3B
:10103000D12C3AC0FAE0CF16D10491F080E1C81665
:10104000D10429F0E8E0CE16D104F9F415C0BFEFC1
:10105000EB2EBFEFFB2EBFEF0B2FBFE01B2F24C0EB
:10106000A9E9EA2EA9E9FA2EA9E90A2FA9E11A2F7E
:101070001BC0F8E0CF2ED12CEFEFEE2EEFEFFE2EBF
:10108000EFEF0E2FEFE11E2F0FC09601442737FD23
:101090004095542F6FEF7FEF8FEF9FEF0E9429361F
:1010A000C901DA017C018D0120E030E040E050E030
:1010B00060E03601882477FC8094982C70EDB72E80
:1010C000BA0CF9E0FB1570F48A2D81548A3118F4BA
:1010D00099ECB92E06C08A2D81568A3148F589EAE5
:1010E000B82EBA0C8B2D90E08C159D050CF56F3F3A
:1010F000E9F0E216F30604071507B8F0CA01B901D2
:10110000A40193010E94F7359B01AC018B2D90E067
:10111000A0E0B0E0280F391F4A1F5B1F28173907CE
:101120004A075B0710F061E001C06FEFA990C6CFDE
:101130004114510451F0662311F0219703C031FE90
:1011400004C02297F201D183C08330FE07C05095BE
:101150004095309521953F4F4F4F5F4F67FF0AC035
:1011600082E290E09093E8068093E7062FEF3FEF4E
:101170004FEF5FEFB901CA01CDB7DEB7E1E10C94E3
:101180008336FC0188279927E89421912032E9F3DE
:10119000293010F02E30C8F32B3241F02D3239F4C3
:1011A000689404C00E941609820F911D219120535A
:1011B0002A30C0F31EF4909581959F4F089540EC1E
:1011C00053E00E94E4080895009731F4DA018D910C
:1011D0009C91009709F40EC0DC01FB013D91219127
:1011E000222319F03217C9F3FACF332331F4DA018D
:1011F0001D921C928827992708951197AF93BF934A
:10120000FB013D912191321771F4332321F488279A
:101210009927119702C01E921196FA01A193B083EB
:101220009F918F910895222369F7EACF7AE0979FE3
:10123000902D879F802D910D112408958091C203D8
:10124000813019F482E08093C2038091C20383301D
:1012500019F484E08093C2030895009721F19C0162
:1012600040E050E068E478EE81E090E00E944B3688
:10127000C901DA018F3F9105A105B10531F028F0D0
:101280008FEF90E0A0E0B0E008C00097A105B105A5
:1012900021F481E090E0A0E0B0E08093D100809163
:1012A000C000806103C08091C0008F7E8093C00029
:1012B0000895EBE6F0E0808180688083E8E6F0E066
:1012C00080818160808308951F920F920FB60F92E4
:1012D00011242F933F934F935F936F937F938F933B
:1012E0009F93AF93BF93EF93FF931F9902C00E9408
:1012F0001E09FF91EF91BF91AF919F918F917F91C7
:101300006F915F914F913F912F910F900FBE0F9072
:101310001F90189581E008951F93182F0E948A0945
:101320008823E9F02FB781E08093CB05F894809172
:101330000008909101088757974709F0A89588E120
:101340008093600010936000112341F080910008A9
:10135000909101088757974709F0A8952FBF1F91D3
:101360000895382F20E080915D0590915E058227D9
:10137000932740E061E270E19C01220F331F97FF49
:1013800004C0C9018627972701C0C9014F5F4830B3
:1013900099F790935E0580935D05089587E38093A8
:1013A000F80380E092ECA1E0B0E08093F903909321
:1013B000FA03A093FB03B093FC0387E0809305043A
:1013C00080EC9AECA9E8B6E38093FD039093FE03CA
:1013D000A093FF03B093000485E0809306048DEE94
:1013E0009EEFADEABEED8093010490930204A093BA
:1013F0000304B0930404A7E0B4E080E090E08630FA
:1014000010F0E0E004C0FC01E657FC4FE081ED93F2
:1014100001968831910599F782E080931F048AE054
:1014200080932004089580EC97EFAAEBB7E38093B4
:10143000C5039093C603A093C703B093C80380E08D
:1014400090E0A0E0B0E58093C9039093CA03A09315
:10145000CB03B093CC03EDECF3E080E081938F5F9E
:101460008031E1F708958436910520F4BC0180E0D5
:1014700090E025C08E3B910550F48A559040BC0108
:1014800080E090E02AE030E040E050E016C0823D8D
:10149000910550F4845B9040BC0180E090E024E62C
:1014A00030E040E050E009C08D5C9040BC0180E03D
:1014B00090E028E532E040E050E00E94F73524E675
:1014C00030E040E050E00E94F735089590E08C59FC
:1014D0009F4F0E94330A0895DC019896EC91F0E04A
:1014E000E770F070EE57FC4F808108958F929F92C5
:1014F000AF92BF92CF92DF92EF92FF920F931F9322
:101500008C010E946C0AD80197962C9130E043E13F
:1015100050E0249FF001259FF00D349FF00D112421
:10152000EB54FD4F80809180A280B38090E00F96B5
:10153000AA2797FDA095BA2FBC01CD0120E43FE179
:101540004DE750E00E94F735A50194010E9429362D
:1015500069017A0180ED97E0A0E0B0E0C80ED91EE5
:10156000EA1EFB1ED80198968C91887181F060E08C
:101570007EEE8AEB9BE0A50194010E94293628515A
:101580003C4F4F4F5F4FC20ED31EE41EF51E87EE39
:1015900093E0A0E0B0E0C80ED91EEA1EFB1EC70112
:1015A000B60128EE33E040E050E00E942936CA013F
:1015B000B90128EE33E040E050E00E94F7351F917A
:1015C0000F91FF90EF90DF90CF90BF90AF909F90E2
:1015D0008F9008958F3F910509F010F480E00895F1
:1015E00022E08030920710F481E00895805093400B
:1015F00010F083E0089582E00895CF92DF92FF9289
:101600000F931F93CF93DF93F82FEB016A01182FED
:101610001695E0E088819981D6018C938A819B811F
:1016200011968C9311978C819D8112968C931297B1
:101630008E819F8113968C931397288139814A81DB
:101640005B816C817D818E819F819295990F990F2D
:10165000907C832F8370982B852F8370880F880F41
:10166000982B872F83708295807F982B14969C935C
:1016700085E090E0C80ED91E2896EF5F1E1750F641
:10168000F0FF21C0888199810E94EA0AF82E8A81A0
:101690009B810E94EA0A182F8C819D810E94EA0A90
:1016A000082F8E819F810E94EA0AF294FF0CFF0CA2
:1016B00070ECF7221295107F1F29182B000F000FD6
:1016C000012BD6010C93DF91CF911F910F91FF90C9
:1016D000DF90CF90089523E08032920718F420E045
:1016E00030E026C023E0883E920748F49C012F5149
:1016F000334054E0369527955A95E1F719C027E015
:10170000803D920720F49C012C5D334011C028E0FD
:101710008839920718F02FEF33E00AC09C01285C4B
:10172000374044E0369527954A95E1F72D503C4FD8
:10173000C90108958C30910548F49C0174E0220F92
:10174000331F7A95E1F7285D3C4F17C023E0843FB3
:10175000920720F49C0124523C4F0FC024E08030BB
:10176000920718F020E938E008C09C012657334F53
:1017700064E0220F331F6A95E1F7C90108959C01C7
:101780003695279525753575821B930B9C013695EB
:101790002795369527952373337383739373280F97
:1017A000391FC901E4E096958795EA95E1F7820F24
:1017B000931F8F709F7021E031E0AC01429FC00108
:1017C000439F900D529F900D1124892F08958823D7
:1017D00039F0299800002A9A0000299A00000895FB
:1017E000299800002A980000299A00000895299A53
:1017F000000083B12998000090E0B3E096958795AA
:10180000BA95E1F7817008950F931F93082F5E9AA0
:1018100029985E9810E0802F80780E94E70B000FD7
:101820001F5F1830C1F729981F910F9108958F7786
:101830000E94040C08950F931F93082F10E0802F2F
:1018400080780E94E70B000F1F5F1830C1F72998BE
:101850001F910F9108950F931F93299880E000E046
:10186000182F110F0E94F70B810F0F5F0830C1F77F
:101870001F910F9108950E94170C0E942B0C5E9AE5
:1018800008951F93162F80680E94040C812F0E94D8
:101890001B0C5E9A1F9108951F9310910104182745
:1018A000E8EFF3E0E80FF11D89E767850E94410C3E
:1018B0008DE3612F0E94410C82E4612F0E94410C54
:1018C0001F91089586E20E943B0C08950F931F9389
:1018D0008C018CE1F80164810E94410C8DE1F801DA
:1018E00065810E94410C8EE1F80166810E94410CE5
:1018F00080E2F80167810E94410C81E2F801608575
:101900000E94410C82E2F80161850E94410C83E251
:10191000F80162850E94410C84E2F80163850E940F
:10192000410C85E2F80164850E94410C8AE2F801CD
:1019300065850E94410C8EE6F80166850E94410C87
:101940008FE6F80167850E94410C80E7F801608905
:101950000E94410C81E7F80161890E94410C82E7F5
:10196000F80162890E94410C1F910F910895EF9236
:10197000FF920F931F93CF93DF937B018C01603015
:1019800028E372072CE982072CE1920728F520E86A
:1019900036E948E950E00E942936E9016897B90123
:1019A00080E090E020E839E647E65FEF0E94F735F7
:1019B0006E0D7F1D801F911F32E0660F771F881FFD
:1019C000991F3A95D1F721E732E040E050E00E94BC
:1019D0002936890180E421C020E03DE241E351E065
:1019E0000E942936E9016897B90180E090E020E083
:1019F00033ED4EEC5EEF0E94F7356E0D7F1D801FBC
:101A0000911F660F771F881F991F21E732E040E082
:101A100050E00E942936890180E69E012F71622FD5
:101A2000680F85E70E94410C86E7612F0E94410CF8
:101A300087E7602F0E94410CCDB7DEB7E6E00C943B
:101A40008E36682F8DE60E94410C08959F92AF92CA
:101A5000BF92CF92DF920F93DF93CF9300D000D04D
:101A6000CDB7DEB7982E83E00E943B0C8093210413
:101A700084E00E943B0C8093220486E060E00E9498
:101A8000410C87E061E00E94410C89E06FE70E9411
:101A9000410C8AE065E00E94410C8BE065E10E9408
:101AA000410C8CE062E10E94410C8DE06DEF0E94E0
:101AB000410C8EE060E00E94410C992019F084E115
:101AC00093E008C080911F0423E1829FC00111248C
:101AD0008B549D4F0E94660C80E36CE80E94410C81
:101AE00082E36FE00E94410C83E362E40E94410CB8
:101AF00084E36AE00E94410C85E36AE20E94410CA3
:101B000086E36DE20E94410C87E364ED0E94410C84
:101B100088E360E00E94410C89E360E00E94410C90
:101B2000992049F065E8A62E61ECB62E61ECC62E30
:101B30006EEDD62E08C0A0900104B0900204C090B3
:101B40000304D09004040AE38D2D9927AA27BB270C
:101B500089839A83AB83BC83802F69810E94410C67
:101B6000802F8B5F69810E94410CDC2CCB2CBA2C1E
:101B7000AA240F5F0E3341F783E46FEF0E94410CFC
:101B800084E46FEF0E94410C85E46FEF0E94410CEA
:101B900086E46FEF0E94410C992019F08DE666E013
:101BA00003C08DE6609105040E94410C89E760E066
:101BB0000E94410C8AE7609106040E94410C83E771
:101BC00060E00E94410C84E760E00E94410C992093
:101BD00029F060EC7AEC89E896E308C06091FD0397
:101BE0007091FE038091FF03909100040E94B70C56
:101BF0000F900F900F900F90CF91DF910F91DF908A
:101C0000CF90BF90AF909F90089587E061E00E94D1
:101C1000410C8EE764E20E94410C88E063E00E9480
:101C2000410C88E060E00E94410C87E065E00E9482
:101C3000410C85E062E00E94410C83E00E943B0C75
:101C40008093210484E00E943B0C80932204089539
:101C5000582F4091C604842F90E0FC01EF70F07083
:101C60009F012F5F3F4F74E0959587957A95E1F737
:101C70002817390751F0EA54FB4F5083842F8F5FA8
:101C80008F70407F842B8093C60408951F920F921B
:101C90000FB60F9211241F932F933F934F935F938F
:101CA0006F937F938F939F93AF93BF93CF93DF9364
:101CB000EF93FF93C0918600D091870020910A0591
:101CC00030910B058091E904882309F062C0BE01C0
:101CD000621B730B2091C9033091CA034091CB035F
:101CE0005091CC0325FD02C07695679589E0653C4F
:101CF0007807B8F1809147031CE1569547953795D1
:101D000027951A95D1F7211531054105510521F483
:101D100021E030E040E050E090E0A0E0B0E02817A3
:101D200039074A075B07D0F4809147038F3FB1F032
:101D300020E00EC0E22FF0E0EE0FFF1FDF01A65102
:101D4000BB4F8D919C91E95DFC4F918380832F5F08
:101D500080914703281770F31092E804109247030C
:101D600018C082E06D3B780760F1809147038031B5
:101D700040F510914703CB010E946B0BE12FF0E07F
:101D8000EE0FFF1FE651FB4F918380831F5F10937F
:101D90004703D0930B05C0930A05FF91EF91DF91A4
:101DA000CF91BF91AF919F918F917F916F915F91F3
:101DB0004F913F912F911F910F900FBE0F901F9049
:101DC00018958FEF80934703E4CF83E080938000E2
:101DD0008AE9809381008091C90386FD05C08091C6
:101DE00081008064809381008FEF9FEF9093890042
:101DF0008093880080916F00806280936F000895C7
:101E00006F3018F086958058089589E0689F802D7E
:101E100011240895882319F460E071E002C063E0A2
:101E200071E089E196E00E943D2F0895A0E0B0E0C6
:101E3000ECE1FFE00C947036182F0E94D62A9B012B
:101E4000AC018091570590915805A0915905B0912A
:101E50005A0569017A01C81AD90AEA0AFB0AD701A8
:101E6000C60189589341A040B04010F01092560529
:101E700020935705309358054093590550935A05C0
:101E80002091E904822F81508230E8F58091560537
:101E9000882309F44FC1813011F482E0BCC1803144
:101EA00008F035C1E82FF0E0E651FB4F10838F5F5B
:101EB00080935605803109F0B0C1ACEEB4E021301A
:101EC00039F41196EC911197E695E6958C9109C03D
:101ED0008D919C911197E92FE695E695E69596955B
:101EE0008795E03140F4F0E090E0EE0FFF1FE95DF0
:101EF000FC4F918380831092E804129684E0AA3FFD
:101F0000B807E9F68AC1233009F004C1809156056B
:101F1000882321F41F3009F080C10CC1883130F4CE
:101F2000E82FF0E0E751FB4F108374C1883109F0CE
:101F3000EEC0112309F0EBC0C0E0D0E00BE010E0F0
:101F4000DE0163E0AA0FBB1F6A95E1F7C09FB001F5
:101F5000C19F700DD09F700D1124FB01E651FB4F06
:101F600080812181922F977095958795FD01EE0FC5
:101F7000FF1FE95DFC4F91838083FB01E551FB4F1F
:101F800030813695369536952181422F4295440F02
:101F9000407E842F832B269526952695922F977029
:101FA00095958795FD01EE0FFF1FE75DFC4F91832F
:101FB0008083FB01E451FB4F808182958695869555
:101FC00083704181942F990F990F292F282B4295C7
:101FD00046954695437082818170880F880F382F0F
:101FE000342B35952795FD01EE0FFF1FE55DFC4F66
:101FF00031832083FB01E251FB4F308136952181F3
:10200000422F479544274795842F832B2695922F5F
:10201000977095958795FD01EE0FFF1FE35DFC4FCF
:1020200091838083FB01E151FB4F308132953F70FA
:102030002181422F4295407F842F832B22952F7040
:10204000922F977095958795FD01EE0FFF1FE15D2B
:10205000FC4F91838083FB01E051FB4F8081881FFF
:102060008827881F4181942F990F292F282B441FDF
:102070004427441F82818370880F382F342B359575
:102080002795FD01EE0FFF1FEF5CFC4F318320838E
:10209000FB01EE50FB4F3081369536952181422F62
:1020A0004295440F440F407C842F832B2695269520
:1020B000922F977095958795AA0FBB1FFD01ED5C38
:1020C000FC4F918380836D507B4FFB0120812295D3
:1020D000269527704181342F330F330F330F832F11
:1020E000822B942F92959695977095958795AB5CDA
:1020F000BC4F11969C938E932196C230D10509F066
:102100001FCF8091000583FD02C01092E804109259
:10211000560583C0243009F080C040915605442301
:1021200059F4183AB1F410925E0510925D0588EAF0
:102130000E94B10981E06FC0413019F410935B0532
:1021400004C0423031F410935C05812F0E94B10924
:102150005DC060915C05262F30E0220F331FE42F15
:10216000F0E0C90102968E179F0734F0433268F7FA
:10217000E951FB4F1083E9CF2D5F3F4F40915D0543
:1021800050915E05E217F30749F4912F80E048274C
:10219000592750935E0540935D0538C0812F90E02C
:1021A0004817590789F580915B05813069F56131E0
:1021B00018F080E180935C05D0905C054AEEE42E37
:1021C00044E0F42E00E010E01BC0F701D081C0E035
:1021D000818190E08C2B9D2B33E0969587953A95E5
:1021E000E1F70E946B0BF801EE0FFF1FE95DFC4F5A
:1021F000918380830F5F1F4F82E090E0E80EF91E0D
:102200000D1518F31092E8041092560580915605AA
:10221000882319F08F5F80935605CDB7DEB7E8E0CD
:102220000C948C36FF920F931F93CF93DF93182F4C
:10223000092FF62E8EE30E94410C212F302FC90169
:10224000EC0110E005C08FE769910E94410C1F5F0F
:102250001F15C8F385E064E00E94410C83E00E94F2
:102260003B0C8093210484E00E943B0C8093220469
:102270000E94D62A6093230470932404809325043B
:102280009093260487E069E00E94410C81E08093EE
:10229000C203CDB7DEB7E5E00C948F360E94121171
:1022A0008091C2038130D9F40E94D62A2091230460
:1022B000309124044091250450912604621B730B35
:1022C000840B950B605A76488140904040F4E8CFEB
:1022D00089E196E067E071E00E943D2F08958091CA
:1022E000C2038130A9F308958FEA96E06EE70E9459
:1022F000F5300895A0E0B0E0E0E8F1E10C946F362D
:102300006C018FEA96E06EE70E94F530760100E0FE
:1023100010E0C0E0D0E0B0E2BB2E0AC008301105EA
:1023200021F49E012095F60120870894E11CF11C00
:10233000F7016081862F8D57823040F48FEA96E056
:102340006DE70E94F530F70160816B258FEA96E01A
:102350000E94F5300115110551F0F70180819E01B1
:10236000280F311DC32FDD27C20FD31FD0700F5F81
:102370001F4F0930110591F6CDB7DEB7E9E00C9497
:102380008B36A9E0B0E0E7ECF1E10C947636382F1B
:10239000E62F8091CB0490E0019664E270E00E9409
:1023A0001636982F8093CB0488E9898380E18A834D
:1023B000913071F0913028F0923099F09330E1F43F
:1023C00016C085E08B8381EF8C832F5F2D8317C030
:1023D0009B8381EF8C8384E6489FC00111249D83F9
:1023E0000EC084E08B8381EF8C833D8308C09B8388
:1023F00081EF8C83ED8303C00E94741104C0CE0171
:1024000001960E947A112996E2E00C9492360F937D
:102410001F93CF93DF93182F092F8FEA96E06EE773
:102420000E94F530212F302FC901EC0110E000E2AD
:1024300088818D57823040F48FEA96E06DE70E94E4
:10244000F5308881802788838FEA96E069910E9421
:10245000F5301F5F193061F78FEA96E06EE70E9452
:10246000F530DF91CF911F910F910895A9E0B0E071
:10247000ECE3F2E10C947636382F8091CB0488237C
:1024800079F48EEF89833A836B83842F90E095955E
:1024900087958C832D83198618861F821E822FC0F4
:1024A0004091C604842F90E09C012F70307054E05E
:1024B000959587955A95E1F78217930721F18DEF4E
:1024C00089831A821B82DE01149620E008C0EA5438
:1024D000FB4F80818D93405F2F5F263069F0842F02
:1024E00090E0FC0134E0F595E7953A95E1F78F70BF
:1024F0009070E817F90759F74093C6042A83CE0174
:1025000001960E9407128091CB0490E0019666E04C
:1025100070E00E9416368093CB042996E2E00C947A
:1025200092369F92AF92BF92CF92DF92EF92FF923C
:102530000F931F93B82EA62ED42EC22E902E0E943B
:10254000D62A7B018C018091B5042091C70430917B
:10255000C8044091C9045091CA048823B1F0D8013D
:10256000C701821B930BA40BB50B815E9E42A0405A
:10257000B04020F12C2DDC1408F42D2D8B2D6A2D6C
:10258000422F292D0E94C11111C0D801C701821B01
:10259000930BA40BB50B81539547A040B04070F04E
:1025A0008B2D6A2D4D2D2C2D0E943612E092C704E2
:1025B000F092C8040093C9041093CA041F910F91AC
:1025C000FF90EF90DF90CF90BF90AF909F900895D5
:1025D000E82FF0E0EC53FC4FE185E03158F4F8943B
:1025E000F0E0EE0FFF1FE95DFC4F0190F081E02D60
:1025F000789413C0E03129F0E13129F0E0E0F2E015
:102600000CC082E001C083E00E94212C892B19F4C8
:10261000ECE0F0E002C0E4EFF3E0CF010895A0E2C7
:10262000B0E0E5E1F3E10C946E368CE00E943B0CE7
:10263000882379F589E196E063E171E00E943D2FFE
:102640005F9A80E00E94260D0E94050E5F9821C0CF
:102650008FEA96E00E94BC30482F8091E9048823DD
:1026600021F0842F0E94160F14C080915405E82F8A
:10267000F0E031969F012F713070319780915305B2
:1026800090E02817390729F0E65DFA4F4083209340
:1026900054058FEA96E00E948230892BC9F680911A
:1026A000E904882339F40CC089E196E00E94792C72
:1026B0000E94160F89E196E00E94522C892BA1F707
:1026C0008091C203843009F08EC00E94D62A6093A4
:1026D000D8047093D9048093DA049093DB046115D5
:1026E00071058105910561F481E090E0A0E0B0E022
:1026F0008093D8049093D904A093DA04B093DB04B8
:102700008091E4049091E50481609093E5048093C6
:10271000E40483E08093C2038FE70E94170C01E278
:1027200015E00E942B0CF80181938F01F5E00A322D
:102730001F07B9F740910C0580912105282F30E043
:10274000842F90E08227932786FF40C080E44827AB
:1027500040930C05C90188739070C89709F510E083
:1027600014C01F5F80912004E12FF0E084FF06C0B9
:10277000EF5DFA4F80810E94280E07C0EF5DFA4F8F
:102780008FEA96E060810E94F530212F30E0809141
:10279000210590E0877090708217930714F716C098
:1027A0002F733070232B91F4809122058093DC04E9
:1027B000809123058093DE04809124058093DF04BB
:1027C000809127058093E6041092E70480915505D7
:1027D000813019F482E0809355058091550583304E
:1027E00011F4109255050E94D62A5B016C0180916C
:1027F000E0049091E104A091E204B091E304009719
:10280000A105B105C9F086017501E81AF90A0A0B9C
:102810001B0BD801C701885B9B40A040B04060F013
:102820000E94620C8093DD041092E0041092E10497
:102830001092E2041092E30488EF93E00E94760A7B
:102840002091D4043091D5044091D6045091D704FE
:1028500086017501E21AF30A040B150BE616F7065A
:102860000807190708F42BC1A092D404B092D5042C
:10287000C092D604D092D7048091000890910108AC
:102880008757974709F0A8958091E8048830A0F011
:102890008091C9039091CA03A091CB03B091CC035E
:1028A000FCE1B695A79597958795FA95D1F700978E
:1028B000A105B10509F0A2C18091E8048F5F809362
:1028C000E804E090D804F090D9040091DA04109163
:1028D000DB04E114F1040105110511F188EF93E027
:1028E0000E94760AAE18BF08C00AD10A6A157B0595
:1028F0008C059D0588F48091C90384FD04C080ED9A
:1029000097E00E942D091092D8041092D9041092D9
:10291000DA041092DB0404C080E090E00E942D09EC
:1029200090910C05907C90930C05009154051091AA
:1029300053050117B1F180915505823091F59058FA
:1029400090930C0588EF93E00E946C0A893010F098
:1029500048E002C0482F415030E013C03F5FA32F32
:10296000B0E0812F90E0FC01E65DFA4F2081FD018F
:10297000E45FFA4F2083A65BBA4F2C930196182F81
:102980001F71341710F4101749F710935305832F54
:10299000895C90910C05892B80930C0530934A0536
:1029A0001AC0209155052430D1F490914A05EBE4EA
:1029B000F5E0ADE0B5E0292F30E02E0F3F1F02C05B
:1029C00081918D93E217F307D9F7995C80910C05FB
:1029D000982B90930C0583E08093550536C0809129
:1029E000CF04823059F4916090930C055F9A0DECFE
:1029F00013E07E010894E11CF11C10C090930C05BB
:102A00005F98222319F481E0809355058091550544
:102A1000833069F784E080935505E9CFF80181910F
:102A20008F010E94E812F701819391937F01F3E0F7
:102A30000D3D1F0799F7809120048770BE016F5FDD
:102A40007F4F4DE055E00E94FD0A469A2091CD044B
:102A50002223A1F090910504992381F08091CE0466
:102A60008F5F8093CE048150821729F41092CE0498
:102A7000892F815001C0892F0E94210D8091CC04A3
:102A80000E944C0C88EF93E00E946C0A682F8CE047
:102A900095E00E941211E091CC04EF5FE093CC042A
:102AA000E83131F0F0E0E850FC4F8785882339F4B5
:102AB0001092CC0404C05F9A89E08093E80480916E
:102AC0002004887171F18091C203823051F58091A8
:102AD000E4049091E504880F991F9093E504809396
:102AE000E40483E08093C2030E94050E0E94D62A6C
:102AF0006093E0047093E1048093E2049093E30414
:102B0000611571058105910561F481E090E0A0E017
:102B1000B0E08093E0049093E104A093E204B093CA
:102B2000E3048091200484FF1EC08091E40490910E
:102B3000E5048E7F0E94BF0B182F8091DC0460910A
:102B4000E6040E94000F082F8091DD04612F0E948F
:102B5000000F282F8091DE046091DF04402F009148
:102B6000C3030E94911246988091CF048130D1F026
:102B7000813020F0823009F047C034C082E10E94E9
:102B8000212C892B09F040C081E08093CF040E9462
:102B9000C82A6093D0047093D1048093D204909398
:102BA000D30432C082E10E94212C892B21F50E949E
:102BB000C82A2091D0043091D1044091D204509180
:102BC000D304621B730B840B950B695E73408040CA
:102BD0009040D0F082E08093CF0480ED97E00E9497
:102BE0002D0912C082E10E94212C892B69F080E01E
:102BF00090E00E942D091092CF0406C08091E80455
:102C0000883009F059CF57CFA096EAE00C948A3665
:102C1000219A229A23988BE060E00E94762B8CE028
:102C200061E00E94762B089588E08093C1008AE0DD
:102C300061E00E94762B8AE060E00E94EE2B08950E
:102C4000ACE1B0E0E6E2F6E10C946E360E94D62AE2
:102C50007B018C0181E00E94260D84E7A82E6E0185
:102C60000894C11CD11CB3E0BB2EA982C60161E04F
:102C70000E944E11B092C2030E94050E6AEF70E0EE
:102C800080E090E00E94FC2A8091C203833009F02A
:102C90007DC089E196E00E94522C892B09F076C014
:102CA0000E94D62A6E197F09800B910B6058734CD5
:102CB000894C914008F06AC0D8CF8FE70E94170C6A
:102CC0000E942B0C843509F05CC089830E942B0C78
:102CD000182F00E01093B4040093B3040E942B0C4F
:102CE000080F111D1093B4040093B3040E942B0C21
:102CF0008093B2040E942B0C8093B104813108F0C0
:102D000040C0FF2407C00E942B0C0F561B4FF80138
:102D10008083F3940F2D10E08091B10490E0880F30
:102D2000991F0817190778F380E78983CE01019668
:102D300061E00E944E1183E08093C2030E94050E61
:102D400062E370E080E090E00E94FC2A8091C20380
:102D50008330A9F08FE70E94170C0E942B0C80355E
:102D600081F489830DED13E00E942B0CF80181930F
:102D70008F01F3E0083F1F07B9F781E003C082E04D
:102D800001C083E06C96EAE00C948A368091C2031D
:102D9000833009F092CFF3CF83E00E943B0C809305
:102DA000210484E00E943B0C8093220487E061E0D0
:102DB0000E94410C6AE070E080E090E00E94FC2AF2
:102DC0000E94050E000008950F931F93082F17C04F
:102DD0005F9A64E670E080E090E00E94FC2A5F98D1
:102DE00064E670E080E090E00E94FC2A1F5F10170C
:102DF00078F36CE271E080E090E00E94FC2A10E041
:102E0000F6CF482F392F25E00DC0F999FECF1FBA14
:102E1000842F932F92BD81BD60BD0FB6F894FA9AAE
:102E2000F99A0FBE215059F0F999FECF842F932FB4
:102E300092BD81BDF89A80B5681739F7089582E090
:102E40000E94E4160895A0E0B0E0E9E2F7E10C94F6
:102E50006736482E562EEE24FF2488249924C0E09D
:102E6000D0E0CC24DD2476E4372E04C055245394DE
:102E7000CC24DD24442069F48091C303839DE001C8
:102E8000112464ECE62E63E0F62E59E1852E912C98
:102E90001DC021E0421671F48091C303839DE001BF
:102EA00011246B9648EFE42E43E0F42E39E2832E92
:102EB000912C0CC032E0431649F423ECE22E23E0BF
:102EC000F22E91E0892E912CC8E1D1E03E016C0CEC
:102ED0007D1C10925E0510925D05E3011BC055201C
:102EE00059F4F999FECFD2BDC1BDF89A80B5F7016A
:102EF000E00FF11F808307C0F701E00FF11FCE0143
:102F000060810E9401170E0D1F1DF80180810E9433
:102F1000B10921969E012619022F10E00815190506
:102F2000F0F2CE015520D9F4F999FECFD2BDC1BD42
:102F3000F89A20B5F999FECF2196D2BDC1BD21974F
:102F4000F89A80B590E0B22EAA248A299B29209174
:102F50005D0530915E052817390759F487CF219612
:102F600060915E050E940117CE0160915D050E948F
:102F7000011780E291E0C80ED91E91EEC91692E0C9
:102F8000D90608F477CF852DCDB7DEB7E1E10C94F3
:102F9000833680E061E00E94231781E061E00E94B7
:102FA0002317089582E061E00E942317089582E0CC
:102FB00060E00E9423178091C303843020F01092B8
:102FC000C3030E94D21708951F93182F0E94D7178A
:102FD0008091C303811731F0143020F41093C303A0
:102FE0000E94D2171F9108951F93182F0E94D62A6E
:102FF0006093C7047093C8048093C9049093CA0473
:103000001093B504112329F440E855E260E070E024
:1030100004C040E051EE60E070E08FEA96E00E946C
:10302000FB2F1F91089589E196E0609128040E948A
:10303000B32C08951F93182F89E196E0612F0E9409
:10304000B32C809128048127809328041F91089530
:103050001F93192F0E941A18812F0E941A181F916E
:103060000895DF92EF92FF920F931F93D82E7B016A
:103070001092280409E116E0C80165EB0E94B32C08
:10308000C80162E60E94B32C8D2D0E941A18C70158
:103090000E9428181F910F91FF90EF90DF900895E4
:1030A00010928F0485E6EAE2F4E0DF011D928A9532
:1030B000E9F708951F93182F8F3711F08830E1F545
:1030C000E0918F04EE2309F455C0E150E0938F04A2
:1030D000F0E0E65DFB4F108289E196E06DE00E9432
:1030E000B32C10E00AC0E12FF0E0E65DFB4F89E170
:1030F00096E060810E94B32C1F5F80918F041817A7
:1031000090F389E196E060E20E94B32C89E196E0B9
:103110006DE00E94B32C10E00AC0E12FF0E0E65D04
:10312000FB4F89E196E060810E94B32C1F5F809184
:103130008F04181790F31CC08B3119F40E9450189B
:103140001FC08D30E9F08A30D9F080918F04843629
:1031500088F489E196E0612F0E94B32C80918F045E
:10316000E82FF0E0E65DFB4F10838F5F80938F04C4
:1031700080E007C089E196E067E00E94A92DF8CFC2
:1031800081E01F9108951F93CF93DF93C7E0D4E0B0
:1031900010E03BC089E196E062E271E00E943A2FC4
:1031A00089E196E0612F4AE050E00E94B72E89E164
:1031B00096E06FE271E00E943A2F699170E080E042
:1031C00090E02091060430E040E050E00E94F735A6
:1031D00020E137E240E050E00E94F735DC01CB010E
:1031E0004091FD035091FE036091FF037091000434
:1031F000480F591F6A1F7B1F89E196E02AE030E0E3
:103200000E947E2E1F5F183119F08881882311F6E5
:10321000DF91CF911F910895EF92FF920F931F932B
:10322000882339F489E196E061ED7AE00E94C72DA8
:103230003BC090E00E94330A24E630E040E050E0DA
:103240000E942936122F032FF42EE52E622F732FA2
:10325000842F952F2AE030E040E050E00E9429368C
:1032600089E196E0BA01A9012AE030E00E946F2EC0
:1032700089E196E06EE20E94A92D612F702F8F2DBB
:103280009E2D2AE030E040E050E00E942936AB015C
:10329000BC0189E196E02AE030E00E946F2E89E1CE
:1032A00096E063E70E94DB2D1F910F91FF90EF9056
:1032B0000895FF920F931F93CF93DF9389E196E0D8
:1032C00067EC7AE00E94882D8091DD03813041F423
:1032D00089E196E06EEA7AE00E94C72DFF246DC076
:1032E000823029F489E196E067E97AE0F5CF84300D
:1032F00029F489E196E063E87AE0EECF853071F752
:1033000089E196E068E77AE0E7CFCF2DD0E0C930D9
:10331000D1051CF06F2D685C02C06F2D6F5C89E1D8
:1033200096E00E94A92D89E196E060E77AE00E948C
:10333000882DBE016F5F7F4F89E196E04AE050E043
:103340000E94132F89E196E065E67AE00E94882DBD
:103350008E0103521C4FD8011196EC91E032F8F423
:1033600089E196E068E57AE00E94882DF801818184
:10337000803130F089E196E063E371E00E943A2FFA
:10338000C352DC4F698170E06F7070706F5F7F4F68
:1033900089E196E04AE050E00E94262F0DC0F0E05F
:1033A000EF70F070EE0FFF1FEE5AFC4F60817181DD
:1033B00089E196E00E943D2FF3948091B204F816C3
:1033C00008F4A3CF89E196E06DE37AE00E94882DAE
:1033D0008091F5030E940C1989E196E062E27AE09F
:1033E0000E94882D8091F6030E940C1989E196E0D5
:1033F00067E07AE00E94882D8091F7030E940C1903
:1034000089E196E06CEE79E00E94882D4091ED0311
:103410005091EE036091EF037091F0034115510557
:103420006105710539F189E196E02AE030E00E94FA
:103430007E2E89E196E069EB79E00E94882D8091EB
:10344000F1030E94660AAB01BC0189E196E02AE023
:1034500030E00E947E2E89E196E065E979E00E94E5
:10346000882D89E196E06091F2034AE050E00E94E5
:10347000C92E06C089E196E06CE879E00E94C72D6C
:1034800089E196E06FE679E00E94882D6091F30370
:103490007091F40389E196E04AE050E00E94A32E87
:1034A00089E196E062E579E00E94882D6091EC0365
:1034B000603450F470E06F5F7F4F89E196E04AE03E
:1034C00050E00E94262F06C089E196E069E479E089
:1034D0000E94C72D89E196E06CE279E00E94882D78
:1034E0008091EB0380FD03C065E371E002C069E3F6
:1034F00071E089E196E00E943D2F89E196E06FE05E
:1035000079E00E94882D8091EB0382700E940A0F5F
:1035100089E196E060EF78E00E94882D8091EB03CE
:1035200084700E940A0F89E196E061ED78E00E94C4
:10353000882D8091EB0388700E940A0FCDB7DEB70B
:10354000E5E00C948F361F93CF93DF9389E196E0EB
:103550006BE17CE00E94882D4091FD035091FE03B9
:103560006091FF037091000489E196E02AE030E069
:103570000E947E2E89E196E065E07CE00E94882D25
:10358000409101045091020460910304709104047D
:1035900089E196E020E130E00E947E2E89E196E00C
:1035A0006FEE7BE00E94882D89E196E06091050432
:1035B0004AE050E00E94C92E89E196E069ED7BE087
:1035C0000E94882D89E196E0609106044AE050E06F
:1035D0000E94C92E89E196E063EC7BE00E94882D71
:1035E000C7E0D4E010E012C0112331F089E196E089
:1035F0006DE371E00E943A2F89E196E069914AE01B
:1036000050E00E94B72E1F5F183119F0888188237F
:1036100059F789E196E00E94B12D89E196E06DEAC3
:103620007BE00E94882D89E196E060911F044AE0CA
:1036300050E00E94C92E89E196E068E97BE00E9493
:10364000882DE0912004F0E0E770F070EE0FFF1F8E
:10365000EE58FC4F6081718189E196E00E943D2F18
:1036600089E196E063E87BE00E94882D8091200448
:1036700090E0887190708830910589F089309105CB
:103680001CF4892B39F01BC08031910569F04897F3
:10369000B1F40FC089E196E06AE77BE00EC089E1F2
:1036A00096E06EE67BE009C089E196E068E67BE0A3
:1036B00004C089E196E06EE57BE00E94C72D89E1B8
:1036C00096E06AE47BE00E94882D4091F9035091D6
:1036D000FA036091FB037091FC0389E196E02AE014
:1036E00030E00E947E2E89E196E061E37BE00E945B
:1036F000882D8091C90380710E940A0F89E196E0AC
:1037000068E17BE00E94882D8091C90380740E944B
:103710000A0F89E196E06FEF7AE00E94882D809190
:10372000C90380720E940A0F89E196E062EE7AE096
:103730000E94882D88EF93E00E94760AAB01BC01BD
:1037400089E196E02AE030E00E946F2E89E196E060
:103750006DED7AE00E94882D88EF93E00E94760A52
:103760009B01AC0160E472E48FE090E00E94293696
:1037700089E196E0BA01A9012AE030E00E946F2EAB
:1037800089E196E06AED7AE00E94C72DDF91CF9142
:103790001F910895EF92FF920F931F937C0109E10F
:1037A00016E0C8016F2D70E04AE050E00E94922EB2
:1037B000C8016EE20E94A92DB70184E07695679555
:1037C0008A95E1F76F707070C8014AE050E00E947E
:1037D000922EC8016EE20E94A92D8FE0E822FF24FC
:1037E000C801B7014AE050E00E94922E1F910F914C
:1037F000FF90EF9008950F931F93CF93DF93209145
:1038000029042F3FA9F589E196E061E576E00E9461
:10381000882D83E793E00E94CA1B89E196E060E36C
:1038200076E00E94882D8091B3049091B4040E94A8
:10383000CA1B89E196E06DEF75E00E94C72D89E112
:1038400096E06AED75E00E94C72D89E196E062EC92
:1038500075E00E94C72D89E196E06DE975E00E9450
:10386000C72D89E196E00E94B12D0E94591969C0C7
:1038700012160CF066C0332727FD30958091B204F4
:1038800090E0821793070CF45CC089E196E068E849
:1038900075E00E94882D60912904772767FD709557
:1038A00089E196E04AE050E00E94262F89E196E007
:1038B0006DE575E00E94882D08E210E03AC0C12F46
:1038C000D0E0CC0FDD1FCF56DB4F288130E0809158
:1038D0002904992787FD909501972817390741F505
:1038E00089E196E06FE371E00E943A2F89E196E06A
:1038F000602F4AE050E00E94B72E89E196E063E431
:1039000071E00E943A2FE981F0E0EF70F070EE0F65
:10391000FF1FEE5AFC4F6081718189E196E00E94A1
:103920003A2F89E196E067E471E00E943A2F0F5F39
:103930001F5F8091B104181710F289E196E00E9490
:10394000B12DDF91CF911F910F910895ACE1B0E0BF
:10395000ECEAFCE10C947036282F809129048F3F0B
:1039600009F042C1822F90E0FC013A97EF36F10551
:1039700008F033C1EA5AFF4F0C949D3689E196E076
:1039800069E471E0AEC089E196E069E471E00E940B
:103990003D2F1CC189E196E065E571E00E943D2F55
:1039A00085E78983DE011296EDEDF3E08BE101906E
:1039B0000D928150E1F7CE0101966CE10E944E110B
:1039C0000E94050E83E08093C20368EC70E080E003
:1039D00090E00E94FC2A8091C203843009F0FDC06F
:1039E0008FE70E94170C0E942B0C8983853509F004
:1039F000F4C089E196E06FE375E00E94C72D89E18C
:103A000096E061E275E00E94C72D89E196E063E0EF
:103A100075E0ACC089E196E06DE671E00E943D2F53
:103A200089E68983CE01019661E00E944E110E94D1
:103A3000050E83E08093C20368EC70E080E090E0C4
:103A40000E94FC2A8091C203843009F0C6C08FE72F
:103A50000E94170C0E942B0C89838E010E5F1F4F52
:103A6000FDE1EF2EF12CEC0EFD1E0E942B0CD80177
:103A70008D938D01AE15BF05C1F7ADEDB3E0FE012D
:103A800032968BE101900D928150E1F78981893462
:103A900009F0A3C089E196E065EE74E00E94C72DAD
:103AA00089E196E067EC74E00E94C72D89E196E019
:103AB00069EA74E05BC089E196E067E871E00E9422
:103AC0003D2F8EEF8093290488C020522750922FDB
:103AD00090538091B204891738F489E196E066E941
:103AE00071E00E943D2F79C0909329046FC084E15A
:103AF0008093290489E196E062E774E037C085E1AC
:103B00008093290489E196E06BE374E02FC086E19D
:103B10008093290489E196E064E074E027C087E19E
:103B20008093290489E196E06AEB73E01FC088E185
:103B30008093290489E196E069EA73E017C089E17E
:103B40008093290489E196E065E973E00FC08AE17A
:103B50008093290489E196E060E873E007C08BE177
:103B60008093290489E196E068E573E00E94C72DFF
:103B700034C089E196E06EE373E00E94C72D809126
:103B8000EB0391E01DC089E196E068E273E00E94DA
:103B9000C72D8091EB0392E013C089E196E063E1C9
:103BA00073E00E94C72D8091EB0394E009C089E186
:103BB00096E068EF72E00E94C72D8091EB0398E0D9
:103BC00089278093EB038FEF809329040E94FB1BCE
:103BD00004C089E196E00E94792C89E196E00E9478
:103BE000522C892BB1F763C1822F0E945A18882367
:103BF00009F45DC180918F04882321F48FEF8093B5
:103C000029044DC18AE294E060E070E040E050E0B9
:103C10000E94C3079B01AC0160912904862F99275C
:103C200087FD9095A92FB92FFC013197EB31F10554
:103C300008F025C1EB53FF4F0C949D36E62FFF276C
:103C4000E7FDF0958091B20490E08E179F070CF489
:103C500016C1DA01C9010197A109B1098097A1052F
:103C6000B10540F0FF2410E008E26F010894C1089C
:103C7000D10826C0E352FC4F822F81508083E7C0D9
:103C8000612F70E0660F771F6F567B4FFB018081BD
:103C900090E08C159D0599F4802F90E0A0E0B0E0B5
:103CA00082179307A407B50749F4F601E352FC4FC6
:103CB000DB0111968C918183FF24F3940F5F1F5FCA
:103CC0008091B1041817E0F2C0C02F3F31054105C3
:103CD000510511F008F0D3C02093F503B8C02F3F71
:103CE00031054105510511F008F0C9C02093F603D4
:103CF000AEC02F3F31054105510511F008F0BFC09E
:103D00002093F703A4C080912A048062803719F5BC
:103D10008BE294E060E070E040E050E00E94C30776
:103D20009B01AC01DC01CB010197A109B109089706
:103D3000A105B10508F0B6C0CA01B90124ED30E310
:103D400040E050E00E94F7359B01AC012A5E3C4AFE
:103D50004A46554E24C0863611F58BE294E060E069
:103D600070E040E050E00E94C3079B01AC01DC0121
:103D7000CB010197A109B1090797A105B10508F089
:103D800091C0CA01B90128EA31E640E050E00E9442
:103D9000F7359B01AC01245E3C434E46544E211541
:103DA00031054105510561F0DA01C901805C9D4989
:103DB000A845B54381509A45A246B24008F05FC07D
:103DC0002093ED033093EE034093EF035093F00301
:103DD0003EC02F3F31054105510511F008F04FC09D
:103DE0002093F10334C0DA01C9010197A109B10997
:103DF0008F3F9105A105B10508F041C02093F20362
:103E000026C0DA01C901845C9940A040B0408D54BD
:103E10009D41A040B04038F43093F4032093F30365
:103E2000FF24F39401C0FF242115310541055105FC
:103E300011F48FEF07C0213431054105510528F4F5
:103E4000822F81508093EC0302C0FF20C1F080914B
:103E500090048823D1F48091010490910204A091F0
:103E60000304B09104040196A11DB11D80930104C7
:103E700090930204A0930304B093040406C089E164
:103E800096E068EA71E00E943D2F0E9450188FEF83
:103E90008093290489E196E06AE00E94DB2D0E946C
:103EA000FB1B05C021E030E040E050E07DCF6C9688
:103EB000E8E00C948C3689E196E06CEA72E00E94AE
:103EC000C72D89E196E064E972E00E94C72D89E17F
:103ED00096E00E94522C892B31F089E196E00E94F5
:103EE000792C0E94A61C0E942016823019F0833083
:103EF00069F405C089E196E066E772E004C089E1F3
:103F000096E06FE572E00E94C72D08958FEF8093D1
:103F10002904109290040E94FB1B0CC089E196E0DA
:103F20000E94522C892B31F089E196E00E94792C75
:103F30000E94A61C809129048E3F81F708958091EC
:103F40002904992787FD9095A92FB92FFC01319657
:103F5000EB30F10508F074C0E052FF4F0C949D3631
:103F600089E196E064EC78E00E94C72D83E793E056
:103F70000E94CA1B89E196E06CEA78E00E94C72D96
:103F800089E196E067E878E00E94C72D89E196E034
:103F90006DE578E00E94C72D89E196E06CE378E05A
:103FA0000E94C72D89E196E06FE078E00E94C72D5E
:103FB00089E196E069EE77E00E94C72D89E196E0FD
:103FC00065EC77E00E94C72D89E196E06EE977E025
:103FD0000E94C72D89E196E00E94B12D0E94A31A8C
:103FE0002FC089E196E061E877E028C089E196E09A
:103FF0006CE577E023C089E196E067E477E01EC0D6
:1040000089E196E068E277E019C089E196E064EE24
:1040100076E014C089E196E06FEC76E00FC089E1AC
:1040200096E06AEB76E00E94C72D89E196E064E7AE
:1040300076E004C089E196E06EE576E00E94C72D47
:104040006AE070E080E090E00E94FC2A04C089E110
:1040500096E00E94792C89E196E00E94522C892BEF
:10406000B1F70895A2E2B0E0E8E3F0E20C9466361E
:104070008E010F5F1F4F80E1D8011D928A95E9F7ED
:1040800089E196E066EC71E00E943D2F0E94CC161B
:1040900020EC3DE948E555E32F8F38A349A35AA307
:1040A00080EC97EFAAEBB7E38B8F9C8FAD8FBE8F21
:1040B00024EF31E040E050E02F8B388F498F5A8F4A
:1040C00090E5C92E93ECD92EE12CF12C80EC482EF2
:1040D0008DE9582E88E5682E85E3782E882499246A
:1040E000540133241E8A1D8A198A1A8A1B8A1C8A43
:1040F000FFC089E196E00E94792C8434B9F08534C0
:1041000030F48332B9F18C3209F0CCC044C083352D
:1041100009F0C8C02F8D38A149A15AA1C901DA01FF
:104120002C013D01882499245401E2C089E196E0E4
:1041300064E40E94A92D89E196E040EC5DE968E520
:1041400075E32AE030E00E94DD2E89E196E06CE222
:104150000E94A92D89E196E040EC57EF6AEB77E3E6
:104160002AE030E00E94DD2E89E196E06CE20E94B8
:10417000DB2DBEC019821A821B821C821D821E8208
:104180001F82188619861A861B861C861D861E8627
:104190001F86188A3AC0339434E0331609F0A8C059
:1041A00069817A818B819C8128EE33E040E050E088
:1041B0000E94F7356F8F78A389A39AA36D817E81C2
:1041C0008F8198850E94F7356B8F7C8F8D8F9E8FA6
:1041D00089859A85AB85BC858F8B988FA98FBA8F7F
:1041E0006D857E858F8598890E94F7356B017C01EE
:1041F00090E2C9169EE4D90690E0E90690E0F9063F
:1042000030F48CE162E30E94410C332471C0A0E3DE
:10421000CA16A5E7DA06A0E0EA06A0E0FA0618F456
:104220008CE162E2F0CFB0E4CB16BCE9DB06B0E093
:10423000EB06B0E0FB0618F48CE166E2E4CFE0E5C3
:10424000CE16E3ECDE06E0E0EE06E0E0FE0618F453
:104250008CE162E1D8CFF0E6CF16FAEEDF06F0E0AF
:10426000EF06F0E0FF0618F48CE165E1CCCF20E723
:10427000C21621E1D20621E0E20620E0F20618F49F
:104280008CE161E0C0CF30EAC31636E8D30631E0F6
:10429000E30630E0F30618F48CE163E0B4CF8CE180
:1042A00065E0B1CFB0ED2B2E280E49E0421500F1AC
:1042B000032D10E0000F111F000F111F81E090E08F
:1042C0008C0F9D1F080F191FD8016D917D918D9145
:1042D0009C912AE030E040E050E00E94F735620D0A
:1042E000711D811D911DF801608371838283938309
:1042F00089E196E00E94522C892B09F0FACE8114B4
:104300009104A104B10489F4C301B2010E94B70C65
:1043100061E070E080E090E00E94FC2AFFEFFE8BFD
:104320001D8A198A1A8A1B8A1C8A2F89388D498D01
:104330005A8D82169306A406B506E0F40E94620C1C
:1043400029893A894B895C89280F311D411D511DEE
:10435000298B3A8B4B8B5C8B3D89381708F48D8BFE
:104360004E89841708F48E8B0894811C911CA11C23
:10437000B11C56C0C301B20128EE33E040E050E06A
:104380000E94293689E196E0BA01A9012AE030E0CD
:104390000E946F2E89E196E06CE20E94A92D89E1CE
:1043A00096E06D894AE050E00E94B72E89E196E0E0
:1043B0006CE20E94A92D69897A898B899C89A50163
:1043C00094010E94293689E196E0BA01A9012AE008
:1043D00030E00E946F2E89E196E06CE20E94A92DE8
:1043E00089E196E06E894AE050E00E94B72E89E1AB
:1043F00096E06CE20E94DB2D4C0C5D1C6E1C7F1C59
:104400008B8D9C8DAD8DBE8D84159505A605B7054C
:1044100020F44F8C58A069A07AA0882499245401D4
:104420002F8D38A149A15AA1285E33404040504009
:1044300009F05ECFA296E2E10C948236A0E0B0E0F3
:10444000E4E2F2E20C9471360E94D62A61157105FD
:1044500081059105C9F30E94BA07109201041092D8
:1044600002041092030410920404DD24E09001047D
:10447000F09002040091030410910404102F0F2DFA
:10448000FE2CEE240E94B5072FEF30E040E050E014
:104490000E944B36E60EF71E081F191FE09201041A
:1044A000F09202040093030410930404D39444E0B4
:1044B000D416E1F6C7E0D4E000E010E020E1E22EFF
:1044C00027E2F22E4EC00F5F19F40E94CE094DC0B4
:1044D0000E94B50722E330E040E050E00E944B36F6
:1044E0006F5FE7E0F4E090E004C08191861759F334
:1044F0009F5F9117D0F38091060490E08E9D90010C
:104500008F9D300D9E9D300D1124862F90E0AC01C3
:10451000249FC001259F900D349F900D1124AA2740
:1045200097FDA095BA2F2091FD033091FE03409195
:10453000FF0350910004820F931FA41FB51F209109
:10454000C5033091C6034091C7035091C803281793
:1045500039074A075B0708F4B6CF69931F5F183124
:1045600021F08881882309F0AECFCDB7DEB7E7E030
:104570000C948D3680E060E00E942317882331F090
:1045800081E060E00E942317882341F40E94130A0F
:104590000E94CE090E941E220E94C9170895AAE512
:1045A000B0E0E5EDF2E20C9472368B017A018B30CB
:1045B00009F426C18C3040F5853009F484C086307A
:1045C00080F4823009F459C0833020F4813009F03E
:1045D00050C242C0833009F461C0843009F049C23E
:1045E00065C0883009F49DC0893038F4863009F4FC
:1045F00086C0873009F03DC28CC0893009F499C06B
:104600008A3009F036C2C9C0893609F482C18A36B7
:1046100080F4863609F42DC1873620F4853609F0FA
:1046200028C20EC1873609F43DC1883609F021C27F
:1046300041C18C3609F4C4C18D3638F48A3609F488
:1046400073C18B3609F015C2AFC18D3609F4ECC1C8
:10465000873C09F00EC200C281E069E270E00E946E
:10466000311808EF13E0F80181918F010E941A18A8
:10467000F4E001321F07B9F704C282E06BE170E099
:104680000E9431180DED13E0F80181918F010E9415
:104690001A18F3E0083F1F07B9F7F3C183E061E0A0
:1046A00070E00E9431180E942016E9C184E061E0A8
:1046B00070E00E94311881E00E941A180E941318BD
:1046C0000E943220E0C16091B10470E0660F771F54
:1046D00085E00E94311800E010E008C0F801EF56B4
:1046E000FB4F80810E941A180F5F1F4F8091B10409
:1046F00090E0880F991F0817190780F3C2C186E060
:1047000062E070E00E94311883E793E00E9428186D
:10471000B8C187E061E070E00E9431188091B20476
:10472000AEC188E061E070E00E9431188091C3035F
:10473000A6C186E68983CE01019661E00E944E11F2
:104740000E94050E83E08093C20368EC70E080E075
:1047500090E00E94FC2A8091C2038430E1F48FE74C
:104760000E94170C0E942B0C8983863471F489E017
:1047700060E270E00E94311810E00E942B0C0E9451
:104780001A181F5F1032C9F77CC189E061E070E040
:104790000E943118C7C089E06DC18AE069E170E00C
:1047A0000E94311882E08093C4038091CB05882356
:1047B00051F08091C9039091CA03A091CB03B091AD
:1047C000CC03806809C08091C9039091CA03A0916D
:1047D000CB03B091CC038F778093C9039093CA0326
:1047E000A093CB03B093CC0304EC13E0F8018191C8
:1047F0008F010E941A18F3E00D3D1F07B9F741C160
:104800008BE061E270E00E9431188091E8048F3FF4
:1048100039F08091E8048F5F8093E804815002C0F2
:104820008091E8040E941A1810E0812F0E94E8127B
:104830000E949A0B0E9428181F5F1031B1F721C106
:1048400085E661E070E00E9431180932110509F037
:1048500015C120E030E0F901E850FC4FD701A20F6C
:10486000B31F8C9180832F5F3F4F2932310599F719
:1048700059C086E661E070E00E9431180B311105E5
:1048800009F0FCC020E030E0F901E352FC4FD70111
:10489000A20FB31F8C9180832F5F3F4F2B313105C7
:1048A00099F740C087E661E070E00E9431180E94ED
:1048B000C91738C088E661E070E00E94311885E7CA
:1048C0008A83DE011396EDEDF3E08BE101900D920A
:1048D0008150E1F7CE0102966CE10E944E110E94D8
:1048E000050E83E08093C20360E273E080E090E015
:1048F0000E94FC2A8091C203843009F0BFC08FE778
:104900000E94170C0E942B0C8A83853509F0B6C0D3
:1049100009C089E661E070E00E9431180E94CE096A
:104920000E94130A81E0ABC08AE661E070E00E9459
:10493000311889E68E8FCE014E9661E00E944E11AD
:104940000E94050E83E08093C20360E273E080E082
:1049500090E00E94FC2A8091C203843009F08EC04E
:104960008FE70E94170C0E942B0C8E8F8E01015E28
:104970001F4F4AE3E42EF12CEC0EFD1E0E942B0C7F
:10498000F80181938F01EE15FF05C1F7ADEDB3E09E
:10499000FE017F968BE101900D928150E1F78E8DA3
:1049A000893409F06BC0BECF8BE661E070E00E94F5
:1049B0003118F70180810E94E4170E94BA22B2CF19
:1049C0008CE661E070E00E9431180032110571F44C
:1049D00087E68AAFDE01DB96F70180E201900D9257
:1049E0008150E1F7CE01CA9661E205C087E48AAF43
:1049F000CE01CA9661E00E944E110E94050E83E02E
:104A00008093C2036CE474E080E090E00E94FC2A92
:104A10008091C203843091F58FE70E94170C0E94A9
:104A20002B0C873459F57ECF8DE661E070E00E9453
:104A300031180931110511F520E030E0F901EC538E
:104A4000FC4FD701A20FB31F8C9180832F5F3F4F84
:104A50002931310599F766CF87EC61E070E00E945B
:104A6000311881E00E941A180E941318109227042E
:104A70000AC08AEC61E070E00E94311880E00E9478
:104A80001A180E941318C65ADF4FE6E00C948E36AF
:104A9000A0E0B0E0EEE4F5E20C946E3684E0A82EDF
:104AA00006E0B02E15E0C12E0FE515E0B4E6DB2ED2
:104AB000A2E0EA2EF3E0FF2EA1C089E196E00E9479
:104AC000792C982F8093CA058091C905833021F1F4
:104AD000843028F4813099F08230B8F409C08530F0
:104AE00009F448C0853020F1863009F087C05FC0E6
:104AF000953B09F083C081E08093C9057FC0923661
:104B000009F07AC0E092C90579C09093C8059093E6
:104B1000C705F092C90572C09093C5051092C605ED
:104B20008091C70589278093C705A092C90566C0F3
:104B3000D92FC0E02091C5053091C6052C2B3D2B07
:104B40003093C6052093C5058091C70589278093BA
:104B5000C705C092C9052536310508F44FC08CEC55
:104B600061E070E00E94311881E00E941A180E94F2
:104B7000131842C02091C3053091C405F901E15AD0
:104B8000FA4F90838091C70589278093C7052F5FCF
:104B90003F4F3093C4052093C3058091C505909184
:104BA000C6052817390750F1B092C90527C0809172
:104BB000C705891759F46091C3057091C4058091A8
:104BC000C8054FE555E00E94CF220DC08BEC62E096
:104BD00070E00E9431188091C8050E941A188091D7
:104BE00028040E941A18F8018D2D11928A95E9F770
:104BF0001092C4051092C3051092C90589E196E090
:104C00000E94522C892B09F058CFCDB7DEB7EAE0CD
:104C10000C948A3681E08093270408C089E196E0ED
:104C20000E94522C892B11F00E9448258091270464
:104C30008823A1F708951F93109129041F3F09F0BD
:104C4000F1C0893409F467C08A3428F5883309F43F
:104C500079C0893368F4803309F486C0813308F061
:104C60006FC08B3109F44DC0813209F0D5C03DC011
:104C7000813409F49AC0823438F4893309F472C05B
:104C8000803409F0C9C031C0823409F4A1C086342F
:104C900009F0C2C052C0823609F49AC0833690F43B
:104CA000883579F1893538F4823509F43FC0833588
:104CB00009F0B2C01FC08A3509F4A9C0813609F0D5
:104CC000ABC073C0823791F1833730F48636A9F1D7
:104CD000893609F0A1C01FC0883799F08A3709F4D6
:104CE00096C0833709F098C005C089E196E069E471
:104CF00071E019C00E94C91789E196E063ED71E087
:104D000006C00E94BA2289E196E06DEE71E00E9431
:104D10003D2F8EEF7FC00E94CE090E94130A89E1C9
:104D200096E06CE072E00E943D2F76C00E941E2249
:104D300089E196E065E272E0F6CF0E94C3186CC08C
:104D4000805368C089E196E06CE472E00E94C72D50
:104D500090912004892F885F8871977E892B80939A
:104D6000200420C089E056C089E196E069E372E042
:104D70000E94C72D8091C9039091CA03A091CB03D3
:104D8000B091CC0320E130E040E050E0822793274F
:104D9000A427B5278093C9039093CA03A093CB039C
:104DA000B093CC031093290437C089E196E063E205
:104DB00072E00E94C72D8091C9039091CA03A0910F
:104DC000CB03B091CC0320E430E040E050E012C0CF
:104DD00089E196E062E172E00E94C72D8091C903EB
:104DE0009091CA03A091CB03B091CC0320E230E0B4
:104DF00040E050E082279327A427B5278093C9037A
:104E00009093CA03A093CB03B093CC0302C00E943B
:104E10005B1F8FEF80932904809129048E3F09F452
:104E2000DDC0D4C00E945A18882309F4D7C08091ED
:104E30008F04882321F48FEF80932904C7C08AE26E
:104E400094E060E070E040E050E00E94C3079B0106
:104E5000AC0180912904992787FD9095A92FB92F3E
:104E6000FC013197E930F10508F08CC0E551FF4FA6
:104E70000C949D36DA01C901815C9D49A845B54372
:104E80008F5F9945A246B24008F07CC02093FD0395
:104E90003093FE034093FF03509300049AC0209385
:104EA000010430930204409303045093040481E00E
:104EB000809390048EC0283031054105510508F0DB
:104EC00061C02093050485C0DA01C9010197A109D9
:104ED000B1090A97A105B10508F054C02093060452
:104EE00078C08AE294E06DE371E00E94DF0810E090
:104EF0000EC0183130F4E12FF0E0E850FC4F878706
:104F00001F5F80E090E06DE371E00E94DF08009792
:104F100059F00E94C108009761F706C0E12FF0E048
:104F2000E850FC4F17861F5F1831C0F352C0253080
:104F300031054105510530F520931F044AC0DA01BF
:104F4000C9010197A109B1090697A105B105D0F4DE
:104F500080912004887F822B809320043AC0DA015C
:104F6000C9010197A109B1098050924CA140B040FC
:104F700048F42093F9033093FA034093FB035093D2
:104F8000FC0327C089E196E068EA71E00E943D2FAA
:104F900013C08091010490910204A0910304B09188
:104FA00004040196A11DB11D809301049093020495
:104FB000A0930304B09304040E9450188FEF8093D1
:104FC000290489E196E06AE00E94DB2D0E949F1F80
:104FD00005C0809190048823E1F2EECF1F910895DF
:104FE0008FEF80932904109290040E949F1F0CC0A1
:104FF00089E196E00E94522C892B31F089E196E0FC
:105000000E94792C0E941B26809129048E3F81F7F3
:105010006AE070E080E090E00E94FC2A04C089E130
:1050200096E00E94792C89E196E00E94522C892B0F
:10503000B1F70895AAE2B0E0E0E2F8E20C946B3632
:105040000E94C82A7B018C0181E00E94260D04C0C9
:1050500089E196E00E94792C89E196E00E94522C29
:10506000892BB1F75F98DD24D39432E6732E22E0CA
:10507000822E912C8C0E9D1E5E010894A11CB11CE9
:1050800093E0C92E0E94C82A20E030E06E197F0903
:10509000800B910B693C71058105910510F021E0B1
:1050A00030E08D2D90E028233923232B99F10E94A5
:1050B000C82A7B018C01469A80ED97E00E942D0959
:1050C0007982D401E8EFF3E089E201900D928150FA
:1050D000E1F7C5016AE20E944E11469880E090E037
:1050E0000E942D09C092C2030E94050E62E370E087
:1050F00080E090E00E94FC2A8091C203843051F449
:10510000C092C2038FE70E94170C0E942B0C8234BE
:1051100009F4DD2482E10E94212C892B49F5DD244C
:10512000D39426C05F9A469A89E196E00E94792C32
:105130008D30910569F08E3091051CF40A97B1F419
:1051400007C08332910569F08234910579F40CC06F
:1051500089E196E064E072E00E94C72D0E94F0278A
:1051600005C00E94322002C00E940A265F9846981D
:1051700089E196E00E94522C892B09F483CFD2CF8B
:105180008F929F92AF92BF92CF92DF92EF92FF9257
:105190000F931F9382E10E94212C892B09F083C079
:1051A00068EC70E080E090E00E94FC2A80E090E0F3
:1051B0000E942D090E94C82A5B016C0140ECE42E7C
:1051C00042E1F42E012D112DE60EF71E081F191FC6
:1051D00006C082E10E94212C892B09F062C00E9446
:1051E000C82A6E157F058007910798F382E10E9417
:1051F000212C892B09F055C080ED97E00E942D09E4
:105200000E94C82A7B018C0199249394882488E405
:1052100096E2A0E0B0E0A80EB91ECA1EDB1E29C0AF
:10522000AE14BF04C006D10638F480ED97E00E94AA
:105230002D09882483941DC00E94C82A6E197F09F5
:10524000800B910B693C71058105910590F00E94DE
:10525000C82A7B018C0180E0992009F481E0982E16
:10526000882319F480E090E002C080ED97E00E946E
:105270002D0982E10E94212C892B91F280E090E09F
:105280000E942D09882049F08091C3038F5F8370AD
:105290000E94E4170E94BA2206C00E941E220E94A9
:1052A000C9170E941A281F910F91FF90EF90DF906D
:1052B000CF90BF90AF909F908F900895EF92FF9204
:1052C0000F931F9380E00E948C090E94081686E0CD
:1052D00061E00E94762B85E061E00E94762B82E1FE
:1052E00060E00E94762B84E060E00E94762B84E0F0
:1052F00061E00E94EE2B0E94141689E196E060E0C6
:1053000070E00E94512C0E94D7170E94BA220E947E
:10531000E50E8FEF8093E8040E94590978940E946B
:10532000C82A7B018C018091E8048F3F09F0DEC020
:105330000E94C82A6E197F09800B910B605D77402F
:105340008040904008F0D2C0EECF89E196E00E9404
:10535000792C89E196E00E94522C892BB1F789E1E2
:1053600096E062E472E00E943A2F83E793E00E94A5
:10537000CA1B89E196E069E572E00E943A2F89E153
:1053800096E066E070E04AE050E00E94262F62E37B
:1053900070E080E090E00E94FC2A89E196E00E94A3
:1053A000522C04970CF189E196E00E94792C82340A
:1053B0009105D1F489E196E00E94792C8E34910513
:1053C00099F489E196E00E94792C8434910561F486
:1053D00089E196E00E94792C819731F480E090E099
:1053E0000E942D090E941A284091F9035091FA0356
:1053F0006091FB037091FC03DB01CA010197A109D5
:10540000B1090497A105B10568F44093E90443305C
:1054100029F040E052EC61E070E004C040EA56E858
:1054200061E070E08FEA96E00E94FB2F0E94C028A6
:105430005F9880E090E00E942D090E94E50E109296
:10544000CD048091C90383FF11C080910D0488238E
:1054500051F080911404882331F080911B0488233B
:1054600011F087E001C085E08093CD0480E00E94C8
:10547000260D8091CC040E944C0C0E94050E1092C7
:105480005305109254051092550510E015C062E3C3
:1054900070E080E090E00E94FC2A80ED97E00E949E
:1054A0002D0962E370E080E090E00E94FC2A80E039
:1054B00090E00E942D091F5F8091C303811738F788
:1054C0008091200490E084FF09C020E088719070F2
:1054D000489709F421E0822F0E94F4178FE00E9480
:1054E0008C091F910F91FF90EF90089580ED97E048
:1054F0000E942D0982E161E00E94EE2B5F9A29CF84
:105500001F920F920FB60F9211242F933F938F93F8
:105510009F93AF93BF938091D0059091D105A091B7
:10552000D205B091D3053091D4050196A11DB11DCE
:10553000232F2D5F2D3720F02D570196A11DB11D72
:105540002093D4058093D0059093D105A093D205E4
:10555000B093D3058091CC059091CD05A091CE0557
:10556000B091CF050196A11DB11D8093CC059093FC
:10557000CD05A093CE05B093CF05BF91AF919F917C
:105580008F913F912F910F900FBE0F901F90189504
:105590008FB7F8942091D0053091D1054091D20574
:1055A0005091D3058FBFB901CA0108959FB7F894F0
:1055B0002091CC053091CD054091CE055091CF057D
:1055C00086B5A89B06C08F3F21F02F5F3F4F4F4FFE
:1055D0005F4F9FBF542F432F322F2227280F311D9B
:1055E000411D511D82E0220F331F441F551F8A9514
:1055F000D1F7B901CA010895EF92FF920F931F935B
:10560000CF93DF937B018C010E94D62AEB010EC061
:105610000E94D62A6C1B7D0B685E7340C8F3089409
:10562000E108F10801091109C851DC4FE114F10446
:105630000105110569F7CDB7DEB7E6E00C948E36AB
:10564000789484B5826084BD84B5816084BD85B55D
:10565000826085BD85B5816085BDEEE6F0E0808124
:1056600081608083E1E8F0E0108280818260808345
:10567000808181608083E0E8F0E0808181608083C8
:10568000E1E9F0E0808182608083808181608083B5
:10569000E0E9F0E0808181608083E1ECF0E08081EE
:1056A0008460808380818260808380818160808348
:1056B000E3ECF0E0808181608083E0ECF0E08081C9
:1056C00082608083E2ECF0E0808181608083EAE7A1
:1056D000F0E080818460808380818260808380812B
:1056E000816080838081806880830895CF93DF9379
:1056F000482F50E0CA018758934FFC013491455A16
:10570000534FFA018491882369F190E0880F991F23
:10571000FC01EF5CF34FA591B491FC01E15CF34F08
:10572000C591D491662351F42FB7F8948C91932F9F
:10573000909589238C93888189230BC0623061F412
:105740002FB7F8948C91932F909589238C9388810F
:10575000832B88832FBF06C09FB7F8948C91832B2F
:105760008C939FBFDF91CF91089590E0FC0131971A
:10577000EE30F10590F5EC50FF4F0C949D36809182
:1057800080008F7703C0809180008F7D80938000A0
:10579000089584B58F7702C084B58F7D84BD089548
:1057A000809190008F7707C0809190008F7D03C01B
:1057B00080919000877F8093900008958091C00031
:1057C0008F7703C08091C0008F7D8093C0000895C3
:1057D0008091C200877F8093C2000895FF920F934B
:1057E0001F93F62E482F50E0CA018956934FFC01B3
:1057F0002491CA018758934FFC011491455A534F85
:10580000FA0104910023C9F0222319F0822F0E948B
:10581000B52BE02FF0E0EE0FFF1FE15CF34FA591F9
:10582000B4919FB7F894FF2021F48C9110958123B7
:1058300002C08C91812B8C939FBF1F910F91FF9081
:1058400008950F931F93482F50E0CA018956934F34
:10585000FC012491CA018758934FFC010491455AD9
:10586000534FFA011491112319F420E030E015C0D0
:10587000222319F0822F0E94B52B812F90E0880FF0
:10588000991F835B934FFC01A591B4918C9120E00B
:1058900030E0802311F021E030E0C9011F910F9129
:1058A00008950895209115063091160680911706E7
:1058B00090911806281B390B2F733070C901089579
:1058C00020911506309116068091170690911806C2
:1058D0002817390719F42FEF3FEF09C0E091170699
:1058E000F0911806EB52FA4F8081282F30E0C90161
:1058F0000895209115063091160680911706909113
:1059000018062817390719F42FEF3FEF13C0E0915D
:105910001706F0911806EB52FA4F20818091170676
:105920009091180601968F7390709093180680934B
:10593000170630E0C901089510921C0610921B064C
:1059400088EE93E0A0E0B0E080931D0690931E06E1
:10595000A0931F06B093200684E993E090931A0663
:10596000809319060895A1E0B0E0E9EBFCE20C9405
:1059700074368C01698380914F03882369F083E03A
:10598000BE016F5F7F4F41E050E00E9490321816D9
:10599000190614F49C0107C081E090E0F80193839C
:1059A000828320E030E0C9012196E4E00C94903637
:1059B00083E00E9467320895CF93DF9312C082E0A4
:1059C0000E94D7312FEF8F3F9207C9F0E091150663
:1059D000F0911606EB52FA4F8083D0931606C093CF
:1059E0001506C0911506D09116062196CF73D0707A
:1059F0008091170690911806C817D90701F7DF9113
:105A0000CF910895FC0180818E5F808380E861ECF6
:105A10007CE042E450E00E940E320895FC01818156
:105A20009081913A59F4813209F04CC080E068E4E9
:105A300073E047E050E00E940E3242C0913209F01C
:105A400041C0803239F488E493E067E070E00E945E
:105A5000523236C0823209F035C0828180934F03C2
:105A60008091480390914903A0914A03B0914B0360
:105A7000805B9440A040B04019F580914F0380FDB9
:105A800012C087E797E790930108809300082BE006
:105A900088E190E00FB6F894A895809360000FBE5F
:105AA000209360000DC088E10FB6F89480936000E9
:105AB000109260000FBEA895109201081092000885
:105AC00081E0089580E00895A0E0B0E0EAE6FDE21C
:105AD0000C9470367C016B018A01C0E0D0E00FC0ED
:105AE000D6016D916D01D701ED91FC910190F0818E
:105AF000E02DC7010995C80FD91F015010400115AD
:105B0000110571F7CE01CDB7DEB7E8E00C948C3605
:105B1000EF92FF920F931F93CF93DF937C018B0142
:105B2000C0E0D0E0F8010F5F1F4F6491662359F089
:105B3000D701ED91FC910190F081E02DC70109950D
:105B4000C80FD91FEFCFCE01CDB7DEB7E6E00C947A
:105B50008E36DC01ED91FC910190F081E02D0995EC
:105B60000895EF92FF920F931F938C016DE00E94B6
:105B7000A92D7C01C8016AE00E94A92D9C012E0D6F
:105B80003F1DC9011F910F91FF90EF900895EF9273
:105B9000FF920F931F937C010E94882D8C01C701F7
:105BA0000E94B12D9C01200F311FC9011F910F913F
:105BB000FF90EF900895EF92FF920F931F937C0157
:105BC0000E94A92D8C01C7010E94B12D9C01200FBC
:105BD000311FC9011F910F91FF90EF900895CF934E
:105BE000DF93EC016115710519F420E030E00FC07E
:105BF000DB010D900020E9F71197A61BB70BE88198
:105C0000F9810280F381E02DAD0109959C01C90164
:105C1000DF91CF9108954F925F927F928F929F92E2
:105C2000AF92BF92CF92DF92EF92FF920F931F93AA
:105C3000DF93CF93CDB7DEB7A1970FB6F894DEBF51
:105C40000FBECDBF2C01742ECB01223008F42AE008
:105C500019A231E2C32ED12CCC0EDD1E822E992446
:105C6000AA24BB24672D752FA50194010E94293613
:105C700079018A01C801B701A50194010E94F73595
:105C8000472D461B0894C108D1084A3010F4405DE6
:105C900001C0495CF6014083E114F10401051105DE
:105CA00021F07E2C5F2DC801DDCFC201B6010E941C
:105CB000EF2DA1960FB6F894DEBF0FBECDBFCF91EA
:105CC000DF911F910F91FF90EF90DF90CF90BF90E9
:105CD000AF909F908F907F905F904F900895DC01E0
:105CE0002115310541F4ED91FC910190F081E02DF9
:105CF000642F099508950E940B2E0895EF92FF924C
:105D00000F931F937C010E946F2E8C01C7010E948C
:105D1000B12D9C01200F311FC9011F910F91FF90E0
:105D2000EF900895EF92FF920F931F939A017B01DA
:105D300000E010E0B801A7010E946F2E1F910F91A3
:105D4000FF90EF900895EF92FF920F931F937C01C5
:105D50000E94922E8C01C7010E94B12D9C01200F40
:105D6000311FC9011F910F91FF90EF900895EF929D
:105D7000FF920F931F939A01E62EFF2400E010E09C
:105D8000B801A7010E946F2E1F910F91FF90EF9015
:105D90000895EF92FF920F931F937C010E94B72EFC
:105DA0008C01C7010E94B12D9C01200F311FC90138
:105DB0001F910F91FF90EF900895A0E0B0E0E3EE07
:105DC000FEE20C947036EC016A017B01211531056D
:105DD00041F4E881F9810190F081E02D642F09956B
:105DE0001BC02A303105B1F477FF13C06DE20E9469
:105DF000A92D8C0144275527BA014C195D096E095C
:105E00007F09CE012AE00E940B2E9C01200F311F3A
:105E100004C02AE00E940B2E9C01C901CDB7DEB759
:105E2000E8E00C948C36EF92FF920F931F937B0166
:105E30009A010027F7FC0095102FB801A7010E94D6
:105E4000DD2E1F910F91FF90EF900895EF92FF923A
:105E50000F931F937C010E94132F8C01C7010E9496
:105E6000B12D9C01200F311FC9011F910F91FF908F
:105E7000EF9008950E94EF2D0895EF92FF920F93F7
:105E80001F937C010E943A2F8C01C7010E94B12D03
:105E90009C01200F311FC9011F910F91FF90EF90BE
:105EA000089508951F920F920FB60F9211242F9309
:105EB0003F934F938F939F93EF93FF938091C800ED
:105EC00082FD1DC04091CE0020916706309168068A
:105ED0002F5F3F4F2F7330708091690690916A0653
:105EE0002817390771F0E0916706F0916806E95DBF
:105EF000F94F4083309368062093670602C0809173
:105F0000CE00FF91EF919F918F914F913F912F91F3
:105F10000F900FBE0F901F9018951F920F920FB603
:105F20000F9211242F933F938F939F93EF93FF939F
:105F30002091AB063091AC068091AD069091AE06F3
:105F40002817390731F48091C9008F7D8093C900EB
:105F500014C0E091AD06F091AE06E559F94F2081ED
:105F60008091AD069091AE0601968F7390709093DC
:105F7000AE068093AD062093CE00FF91EF919F91E6
:105F80008F913F912F910F900FBE0F901F901895FA
:105F9000A0E0B0E0EEECFFE20C946C36FC01138262
:105FA000128288EE93E0A0E0B0E084839583A6831C
:105FB000B78386EA93E091838083758764875787E8
:105FC0004687318B208B138B028BF58AE48AD78A24
:105FD000C68AB18EA08E938E828E8F85848F88899B
:105FE000858F8989868F8A89878F8B8980A3209660
:105FF000ECE00C948836AF92BF92DF92EF92FF9262
:106000000F931F93CF93DF93EC017A018B01DD2473
:10601000403081EE580780E0680780E0780711F093
:10602000DD24D39491E0A92EB12CEC89FD89DD20EB
:1060300069F0C50108A002C0880F991F0A94E2F711
:10604000808360E079E08DE390E005C0108260E835
:1060500074E88EE190E0A80197010E942936215052
:10606000304040405040569547953795279580E100
:106070002030380720F0DD2011F0DD24D6CFE8896C
:10608000F9893083EA89FB89208319A2EE89FF8987
:10609000408121E030E0C9010C8C02C0880F991FBB
:1060A0000A94E2F7482B4083EE89FF894081C901B9
:1060B0000D8C02C0880F991F0A94E2F7482B408389
:1060C000EE89FF894081C9010E8C02C0880F991F9B
:1060D0000A94E2F7482B4083EE89FF8980810F8C78
:1060E00002C0220F331F0A94E2F720952823208351
:1060F000DF91CF911F910F91FF90EF90DF90BF90B4
:10610000AF900895DC011C96ED91FC911D97E05C29
:10611000FF4F2191319180819181281B390B2F7381
:106120003070C90108958FEA96E00E948230892B71
:1061300011F00E94512F0895DC011C96ED91FC9105
:106140001D97E05CFF4F20813181E054F040DF017A
:10615000AE5BBF4F8D919C9111972817390719F4A9
:106160002FEF3FEF07C08D919C91E80FF91F8081C1
:10617000282F30E0C9010895DC011C96ED91FC91B7
:106180001D97E05CFF4F20813181E054F040DF013A
:10619000AE5BBF4F8D919C9111972817390719F469
:1061A0002FEF3FEF10C08D919C911197E80FF91FD1
:1061B00020818D919C91119701968F73907011960B
:1061C0009C938E9330E0C9010895DC0191968C91E7
:1061D0009197882339F05496ED91FC9155978081E1
:1061E00086FFF9CF91961C920895CF93DF93EC012F
:1061F000EE85FF85E05CFF4F20813181E054F04067
:106200002F5F3F4F2F733070DF01AE5BBF4F8D911B
:106210009C91119728173907D1F3E05CFF4F8081DB
:106220009181E054F040E80FF91F6083EE85FF850F
:10623000E05CFF4F31832083EE89FF89208181E07C
:1062400090E00F8C02C0880F991F0A94E2F7282B68
:10625000208381E089A3EC89FD898081806480832B
:1062600081E090E0DF91CF9108958F929F92AF925D
:10627000BF92CF92DF92EF92FF920F931F9300D0C5
:1062800000D00F92EDB7FEB7319684E0ADB7BEB740
:1062900011968C9383E0818387E0828385E08383FA
:1062A00081E084838FEA96E067E276E04BE656E091
:1062B0002DEC30E00CEC10E0B8ECEB2EF12CA9EC5E
:1062C000CA2ED12CFAECAF2EB12CEEEC8E2E912CE6
:1062D0000E94C82F0F900F900F900F900F901F915A
:1062E0000F91FF90EF90DF90CF90BF90AF909F9075
:1062F0008F900895CF93DF930E94202B89ED96E035
:106300000E9472320E945E29C3E9D0E30E940F13FB
:106310002097E1F30E949330F9CFFC0104C08091F3
:10632000F100819361506623D1F7289884E6809329
:10633000D20608959FB7F89487708093E900809102
:10634000F2009FBF0895282F8091D3068823C1F0C3
:1063500057FF1AC015C028989093D2068091F1007B
:106360008193E217F307B9F74115510539F0809190
:10637000F200882319F48BE68093E800AFBF02C0D7
:106380004FEF5FEFCA010895AFB7F89427702093DD
:10639000E9008091F200282F30E0241735070CF433
:1063A000A901FB019B01240F311D94E6DACFA1E086
:1063B000B0E0EDEDF1E30C947636BE016F5F7F4FF8
:1063C00041E050E00E94A331019719F02FEF3FEF19
:1063D00003C08981282F30E0C9012196E2E00C94A6
:1063E00092362FB7F89487708093E9008091E80087
:1063F00085FD02C090E004C08091F20090E4981BFB
:106400002FBF892F08951092E9001092D50610929F
:10641000D4069093D7068093D6060895FF920F93E3
:106420001F93F82E142F052F4091D6065091D706B2
:10643000212F302FC901DC01FB016EEF29C0F7FECF
:1064400002C0949101C090812091D4063091D5066C
:1064500024173507ACF48091E8008570E1F3809152
:10646000E80082FF03C02FEF3FEF17C09093F100C9
:10647000C90101968F739070892B11F46093E80025
:106480002F5F3F4F3093D5062093D4061197319656
:106490001097A9F6812F902F9C01C9011F910F9190
:1064A000FF9008950F931F939C01162F072F809143
:1064B000E80082FFFCCFC901612F0E948D318BEF74
:1064C0008093E800812F902F1F910F910895809362
:1064D000E9008091F200882319F08AE38093E800B4
:1064E000089508951092D30681E08093D70080EA42
:1064F0008093D80082E189BD09B400FEFDCF61E040
:1065000070E080E090E00E94FC2A80E98093D8004F
:106510008CE08093E2001092E000559A209A089552
:10652000A0E0B0E0E6E9F2E30C946A36E82E942E9F
:10653000852E8091D306882309F18B01242F352FD6
:10654000C901EC016AEFF62E57E0752E7E208E2DE4
:1065500090E040E2A42EB12CA822B9223AE3632EA7
:1065600020E4C22ED12CC822D9224CC08E2D0E94EC
:10657000F131282F882361F4FA9419F42FEF3FEFBB
:106580004CC061E070E080E090E00E94FC2A3AC0DC
:1065900090E0C817D9070CF42C2FC21BD1094FB7B4
:1065A000F8947092E900A114B10421F406C010928D
:1065B000F10021502223D9F719C0E7FC03C0F801EC
:1065C000922F10C0C801322F06C0FC010196E49141
:1065D000E093F10031503323C1F706C081918093DD
:1065E000F10091509923D1F7020F111D8091E8001D
:1065F00085FF05C0209729F4C114D10411F06092E1
:10660000E8004FBF209709F0B1CF5D9884E68093F2
:10661000D106292D382DC9019C01C901CDB7DEB79E
:10662000EEE00C9486361F920F920FB60F92112453
:106630002F933F934F935F936F937F938F939F938A
:10664000AF93BF93EF93FF938091E1001092E1002D
:10665000982F93FF0FC01092E90081E08093EB0028
:106660001092EC0082E38093ED001092D30688E054
:106670008093F00092FF28C083E00E94673282E09E
:106680000E949A31882321F089E196E00E94DC2C57
:106690008091D106882351F08091D106815080935A
:1066A000D1068091D106882309F45D9A8091D206A3
:1066B000882351F08091D20681508093D206809138
:1066C000D206882309F4289AFF91EF91BF91AF91E8
:1066D0009F918F917F916F915F914F913F912F91FA
:1066E0000F900FBE0F901F901895A1E0B0E0EBE760
:1066F000F3E30C94743619828E010F5F1F4FC801AB
:106700000E94022DC8010E94EB35898190E02196FC
:10671000E4E00C9490361F920F920FB60F92112462
:10672000CF92DF92EF92FF920F932F933F934F936D
:106730005F936F937F938F939F93AF93BF93EF93E9
:10674000FF93DF93CF93CDB7DEB76197DEBFCDBFA9
:106750001092E9008091E80083FFEBC0CE01019622
:1067600068E00E948D3182EF8093E800998197FF65
:1067700005C08091E80080FFFCCF03C08EEF8093BE
:10678000E800292F30E0C90180769070892B09F04C
:10679000B1C08A81882329F41092F1001092F1008F
:1067A000BDC0813009F4BAC0833009F4B7C0853068
:1067B00049F48091E80080FFFCCF8B818068809352
:1067C000E300ACC0863009F06BC00C81EF80F88428
:1067D000023071F580E090E00E9403320E94753330
:1067E00099E079E0C72ED12CCC0EDD1EF601292FC1
:1067F00011922A95E9F799870A8791E09E8790E898
:10680000988B9AEF998B2091D4063091D506275F0B
:106810003F4F3C872B878D87C7010E94033280E062
:10682000B60149E050E00E940E320E94753376C0F6
:10683000C7010E940332023241F482E290E00E94DA
:10684000E335892B09F46EC069C0013079F48F817A
:106850009885089719F481E08093D8068091D8062E
:10686000882309F063C0E1E4FDE013C0033009F0C0
:1068700059C08B81882319F4E3E0FDE00AC082301F
:1068800019F4E7E0FDE005C0813009F04BC0E9E212
:10689000FDE0449180E8BF0150E00E940E323EC00E
:1068A000873009F43FC0883021F481E08093F10003
:1068B00035C0893099F523703070232B99F5E6E6C1
:1068C000FDE091E031E026E39093E9003093EB00A6
:1068D00084918093EC002093ED009F5F319695307A
:1068E00099F78EE78093EA001092EA008B818093FB
:1068F000D30614C08F8198850E9403328D8188232E
:1069000029F4CE0101960E940E2D06C0823051F46A
:10691000CE0101960E94B434882321F08EEF80933B
:10692000E80007C081E28093EB0003C0E3E5FDE0EF
:10693000B0CF6196DEBFCDBFCF91DF91FF91EF91D8
:10694000BF91AF919F918F917F916F915F914F9187
:106950003F912F910F91FF90EF90DF90CF900F908C
:106960000FBE0F901F901895FC0191818081813A94
:1069700031F4913089F080E0933089F40DC0813298
:1069800069F49B3021F482818093500305C09A30D2
:1069900029F482818093510381E0089580E0089575
:1069A000FC0110820895FC011382128286EB93E0B1
:1069B000918380830895EF92FF920F931F938C0130
:1069C000E62EDC01ED91FC910480F581E02D099526
:1069D000F82ED801ED91FC910680F781E02DC801D9
:1069E0006E2D09958F2D90E01F910F91FF90EF90E4
:1069F00008958AED96E00E94D0348BED96E00E94D7
:106A0000D3340895A1E0B0E0E8E0F5E30C947236E9
:106A100089838B017A0184E0BE016F5F7F4F41E083
:106A200050E00E94903284E4B801A7010E949032A5
:106A30002196E6E00C948E3682E048E050E00E9419
:106A400002350895FC01168217821086118612867F
:106A5000138614823496BF010E941C350895DC0110
:106A6000683810F0685829C0E62FF0E067FF13C0BF
:106A7000E058F04081E090E002C0880F991FEA954D
:106A8000E2F7809514962C911497282314962C9352
:106A9000149760E012C0E851F24F6491662319F434
:106AA00020E030E01DC067FF08C014968C91149759
:106AB0008D7F14968C9314976F77FD0190E0662379
:106AC00021F08681861709F416829F5F31969630F1
:106AD000B1F7CD011496BD010E941C3521E030E0D4
:106AE000C9010895CF93DF93DC01683810F068582E
:106AF00025C0E62FF0E067FF12C0E058F04081E0CB
:106B000090E002C0880F991FEA95E2F714962C9145
:106B10001497282B14962C93149760E00FC0E8511B
:106B2000F24F64916623D9F167FF08C014968C91E7
:106B30001497826014968C9314976F7716968C91A5
:106B400016978617A9F117968C911797861781F1DA
:106B500018968C911897861759F119968C91199758
:106B6000861731F11A968C911A97861709F11B96A0
:106B70008C911B978617E1F0ED01E0E0F0E09E2F8D
:106B80008E81882321F4EA0FFB1F668306C09F5F76
:106B900031962196E630F10591F7963049F481E07F
:106BA00090E013969C938E93129720E030E007C0FC
:106BB000CD011496BD010E941C3521E030E0C901D1
:106BC000DF91CF91089580E86AE67DE045E650E0E8
:106BD0000E940E320895FC0180818F5F808380E8DF
:106BE0006FEC7DE049E150E00E940E320895629F13
:106BF000D001739FF001829FE00DF11D649FE00DB5
:106C0000F11D929FF00D839FF00D749FF00D659F15
:106C1000F00D9927729FB00DE11DF91F639FB00D14
:106C2000E11DF91FBD01CF011124089597FB092E25
:106C300007260AD077FD04D086D006D000201AF4AB
:106C4000709561957F4F0895F6F7909581959F4FC8
:106C50000895A1E21A2EAA1BBB1BFD010DC0AA1F9D
:106C6000BB1FEE1FFF1FA217B307E407F50720F0B5
:106C7000A21BB30BE40BF50B661F771F881F991F30
:106C80001A9469F760957095809590959B01AC0179
:106C9000BD01CF01089597FB092E05260ED057FDA3
:106CA00004D0D7DF0AD0001C38F4509540953095B9
:106CB00021953F4F4F4F5F4F0895F6F79095809580
:106CC000709561957F4F8F4F9F4F08952F923F9200
:106CD0004F925F926F927F928F929F92AF92BF92EC
:106CE000CF92DF92EF92FF920F931F93CF93DF9398
:106CF000CDB7DEB7CA1BDB0B0FB6F894DEBF0FBEF5
:106D0000CDBF09942A88398848885F846E847D8441
:106D10008C849B84AA84B984C884DF80EE80FD8043
:106D20000C811B81AA81B981CE0FD11D0FB6F894B9
:106D3000DEBF0FBECDBFED010895EE0FFF1F059022
:106D4000F491E02D0994AA1BBB1B51E107C0AA1FB7
:106D5000BB1FA617B70710F0A61BB70B881F991FFC
:106D60005A95A9F780959095BC01CD010895911190
:106D700006C0803219F089508550D0F708959927C0
:086D800088270895F894FFCF65
:106D88004E6F005965730054582074696D656F75AE
:106D98007421006D6F64756C65206C6F636B65643E
:106DA8003F00486F70206368616E6E656C2000203C
:106DB80040200053004E2F4100386368002C002CFF
:106DC800205B005D20280029004E4F5420454E418D
:106DD800424C45440053656E64696E672073657460
:106DE80074696E677320746F2052580A0052657375
:106DF800657474696E672073657474696E6773204F
:106E08006F6E2052580A0041626F72746564206583
:106E1800646974730A00696E76616C6964207365CD
:106E28006C656374696F6E000D0A496E76616C69F2
:106E38006420696E707574202D20646973636172B3
:106E48006465642107007363616E6E6572206D6FFF
:106E580064650053657474696E6773207361766541
:106E68006420746F20454550524F4D0A0052657694
:106E780065727465642073657474696E67732066DF
:106E8800726F6D20454550524F4D0A004C6F61643A
:106E9800656420666163746F7279206465666175E4
:106EA8006C74730A004B657920616E6420636861B5
:106EB8006E6E656C732072616E646F6D697A65645D
:106EC8000A004F70656E4C52536E672054582073F9
:106ED80074617274696E672000206F6E20485720B5
:106EE8000050504D005253534900534441005343FE
:106EF8004C00525844005458440041494E004C42FA
:106F08004545500053504B54524D00534255530081
:106F180053554D44004C4C494E440000342B34002A
:106F28003800382B340031320031322B34003136FE
:106F38000001000000C01200001A400AA1204EA55E
:106F4800001B1E27522C23308025000005400AA173
:106F5800204EA50020244EA52C2330004B0000060F
:106F6800400AD0009D49007B289D492C233000E130
:106F7800000005400A4501D7DC03B81E0EBF0023F8
:106F88002E48E801008A400A6001555502AD1E20CE
:106F9800000023C88025000005400AA1204EA50056
:106FA80020244EA52C23300002000200020002001B
:106FB80002000200020002000200020002000200B9
:106FC80002000200020002FF00E1000000000000D1
:106FD8000101610265026A026E02720276027A0299
:106FE8007E0284028B02900295029B029B029B0206
:106FF8009B0235019C02A002A202A602A902AE02CF
:10700800350100070B0C10111500160A132231293F
:1070180000000000B32C642D522C792C602CD82C45
:10702800DC2C00000000F530642D8230BC309C3030
:10703800E53000000000DB34642D72352F35223531
:00000001FF
